:100000000C9422060C944A060C944A060C944A0658
:100010000C944A060C944A060C944A060C944A0620
:100020000C944A060C944A060C944A060C944A0610
:100030000C944A060C944A060C944A060C944A0600
:100040000C944A060C944A060C94E83D0C944A061B
:100050000C944A060C944A060C944A060C944A06E0
:100060000C944A060C944A060C94543C0C944A0690
:10007000687474703A2F2F72617973686F62627955
:100080002E6E65742F736372697074732F6A617654
:10009000612F737663322E3000485454502F312E26
:1000A0003020323030204F4B0D0A436F6E74656E36
:1000B000742D547970653A20746578742F68746D66
:1000C0006C0D0A507261676D613A206E6F2D63612D
:1000D0006368650D0A0D0A003C6D657461206E61F0
:1000E0006D653D76696577706F727420636F6E74AD
:1000F000656E743D2277696474683D363430223E03
:100100000D0A00485454502F312E30203430312005
:10011000556E617574686F72697A65640D0A436F14
:100120006E74656E742D547970653A2074657874B8
:100130002F68746D6C0D0A0D0A3C68313E34303105
:1001400020556E617574686F72697A65643C2F68BA
:10015000313E0077696E646F772E6C6F63617469EE
:100160006F6E3D222F223B3C2F7363726970743E89
:100170000A006376007670006D7000647000637032
:1001800000677000766F00636F00736E007073001D
:10019000767300637300767200637200706E0024E1
:1001A000460024440024440024460024463C6D6557
:1001B000746120687474702D65717569763D227262
:1001C0006566726573682220636F6E74656E743D38
:1001D00022313B2075726C3D2F223E0024463C7339
:1001E00063726970743E616C65727428224F70741A
:1001F000696F6E732076616C7565732073617665C7
:10020000642E22293B24460024463C7363726970A5
:10021000743E616C65727428224E6577207061733C
:1002200073776F726473206D757374206D6174637E
:10023000682122293B77696E646F772E6C6F63614A
:1002400074696F6E3D222F766F223B3C2F73637271
:100250006970743E0A0024463C7363726970743E90
:10026000616C65727428224E6577207061737377B4
:100270006F7264207365742E22293B244600244645
:100280003C7363726970743E616C657274282256A7
:10029000616C756573206F7574206F6620626F7571
:1002A0006E642122293B77696E646F772E6C6F63D1
:1002B0006174696F6E3D222F766F223B3C2F736312
:1002C000726970743E0A0024463C736372697074EC
:1002D0003E2446005265626F6F74696E672E2E2E43
:1002E0000024463C6D65746120687474702D6571DE
:1002F0007569763D22726566726573682220636F48
:100300006E74656E743D2224443B2075726C3D2FE3
:10031000223E003C736372697074207372633D22E5
:1003200024462F766965776F7074696F6E732E6AD5
:1003300073223E3C2F7363726970743E0A003C2F37
:100340007363726970743E0A00305D3B766172209F
:100350006E6F7074733D24442C6C6F633D22245384
:10036000223B00222446222C24442C24442C2444C6
:100370002C003C7363726970743E766172206F70FA
:1003800074733D5B0024462446003C7363726970BD
:1003900074207372633D2224462F686F6D652E6A48
:1003A00073223E3C2F7363726970743E0A003C7383
:1003B0006372697074207372633D22706E2E6A736B
:1003C000223E3C2F7363726970743E0A000A7661A4
:1003D00072206C72756E3D5B24442C24442C2444A2
:1003E0002C244C5D3C2F7363726970743E0A005B71
:1003F000302C305D5D3B0A76617220656E3D244491
:100400002C72643D24442C72733D24442C6D6D3D4C
:1004100024442C726473743D244C2C6D61733D2410
:10042000442C7572733D24442C776C3D24442C6914
:100430007061733D24442C6C6F633D222453223B36
:10044000005B24442C244C5D2C00305D3B766172B3
:100450002070733D5B0024442C00766172206E6234
:1004600072643D24442C747A3D24442C7362697474
:10047000733D5B003C7363726970743E76617220F9
:100480007665723D24442C646576743D244C3B0AA9
:1004900000244624460077696E646F772E6C6F6384
:1004A0006174696F6E3D222F7670223B3C2F73631F
:1004B000726970743E0A00616C6572742822507211
:1004C0006F6772616D202444206D6F646966696591
:1004D0006422293B00616C65727428224E65772086
:1004E00070726F6772616D2061646465642E222989
:1004F0003B0024463C7363726970743E003C736336
:1005000072697074207372633D2224462F706C6F81
:100510007470726F672E6A73223E3C2F7363726928
:1005200070743E0A003C7363726970742073726366
:100530003D22706E2E6A73223E3C2F736372697087
:10054000743E0A00305D3B0024442C00766172202A
:100550006D61736F703D5B0024463C73637269701C
:10056000743E766172207365713D24442C6D617315
:100570003D24442C776C3D24442C7364743D244406
:100580002C6D746F6E3D24442C6D746F66663D2433
:10059000442C6465766461793D24442C6465766DF1
:1005A000696E3D24442C64643D24442C6D6D3D24CF
:1005B000442C79793D24443B0024463C73637269A2
:1005C00070743E77696E646F772E6C6F63617469C7
:1005D0006F6E3D222F7670223B3C2F7363726970E1
:1005E000743E0A003C736372697074207372633DD9
:1005F0002224462F6D6F6470726F672E6A73223EDD
:100600003C2F7363726970743E0A003C2F736372EF
:100610006970743E0A3C736372697074207372630C
:100620003D22706E2E6A73223E3C2F736372697096
:10063000743E0A005D3B002C2444007661722070F9
:10064000726F673D5B24442C24442C24442C2444A6
:100650002C24442C24442C2444003C736372697081
:10066000743E766172206E626F617264733D2444E1
:100670002C7069643D24442C697061733D24443BB3
:100680000024462446003C736372697074207372C0
:10069000633D2224462F7669657770726F672E6AF4
:1006A00073223E3C2F7363726970743E0A003C7380
:1006B0006372697074207372633D22706E2E6A7368
:1006C000223E3C2F7363726970743E0A00244624F4
:1006D000463C7363726970743E0024463C736372D7
:1006E0006970743E2446003C7363726970742073B1
:1006F00072633D2224462F76696577726F2E6A7386
:10070000223E3C2F7363726970743E0A003C73632F
:1007100072697074207372633D22706E2E6A732248
:100720003E3C2F7363726970743E0A00305D3B3C3F
:100730002F7363726970743E0A0024442C002446AF
:1007400024463C7363726970743E766172206E62F7
:100750006F617264733D24442C6D61733D24442C9D
:10076000697061733D24442C6475723D5B003C7379
:100770006372697074207372633D707324442E6ACF
:10078000733E3C2F7363726970743E0A003C2F7392
:1007900063726970743E0A00766172206E70726FC7
:1007A00067733D24442C6E626F617264733D244410
:1007B0002C697061733D24442C6D6E703D24442C73
:1007C00070643D5B5D3B002446005D3B002C24448F
:1007D0000070645B24445D3D5B24442C24442C2441
:1007E000442C24442C24442C24442C24440024460B
:1007F0003C7363726970743E616C65727428224345
:1008000068616E6765732073617665642E22293B8B
:1008100024460024467661722000305D3B3C2F73F5
:1008200063726970743E0A3C7363726970742073FA
:1008300072633D2224462F7669657773746174690B
:100840006F6E732E6A73223E3C2F736372697074ED
:100850003E0A0024442C00766172206D61736F7033
:100860003D5B0024463C7363726970743E7661722E
:10087000206E626F617264733D24442C6D61786CEC
:10088000656E3D24442C6D61733D24442C69706178
:10089000733D24442C0027275D3B0A00272453275F
:1008A0002C00736E616D65733D5B00436F6E6E650A
:1008B0006374696E672E2E2E004669726D776172C1
:1008C00065207665722E0054696D65207A6F6E65BD
:1008D0003A004E54502053796E633A0055736520A8
:1008E000444843503A005374617469632E6970310F
:1008F0003A006970323A006970333A006970343AEC
:1009000000476174657761792E6970313A006970CA
:10091000323A006970333A006970343A00485454EE
:100920005020706F72743A00004175746F207265C8
:10093000636F6E6E6563743A004578702E20626F47
:10094000617264733A0053657175656E7469616CA8
:100950003A0053746174696F6E2064656C61793A12
:10096000004D61737465722073746174696F6E3ABF
:10097000004D61732E206F6E2061646A2E3A004D27
:1009800061732E206F66662061646A2E3A0055738B
:1009900065207261696E2073656E736F723A004EE6
:1009A0006F726D616C6C79206F70656E3A00576183
:1009B000746572696E67206C6576656C3A00536584
:1009C0006C66746573742074696D653A0049676E6E
:1009D0006F72652070617373776F72643A0044655B
:1009E000766963652049443A004C434420436F6E66
:1009F00074726173743A004C4344204261636B6CBF
:100A0000696768743A00526573657420616C6C3F65
:100A1000004D6F6E0054756500576564005468752D
:100A200000467269005361740053756E002073654F
:100A3000630025004E6F00596573002B002B0020CA
:100A4000474D54003030003A002D002B000020208C
:100A50002020002D5261696E2053746F702D002D7F
:100A600044697361626C6564212D003A0045004D54
:100A7000433A003A002E002D0020002020003A00CA
:100A8000200042333A686F6C6420746F2073617683
:100A9000650042333A73656C2042312F42323A632B
:100AA0006867003D3D536574204F7074696F6E73C5
:100AB0003D3D00506C6561736520576169742E2E51
:100AC0002E00526573657474696E672045455052F7
:100AD0004F4D00000108000604000145000082009F
:100AE00000400020504F5354202446204854545076
:100AF0002F312E310D0A486F73743A2024460D0AA7
:100B0000244624534163636570743A202A2F2A0DCA
:100B10000A436F6E6E656374696F6E3A20636C6F23
:100B200073650D0A436F6E74656E742D4C656E6748
:100B300074683A2024440D0A436F6E74656E742DF8
:100B4000547970653A206170706C69636174696F83
:100B50006E2F782D7777772D666F726D2D75726C8D
:100B6000656E636F6465640D0A0D0A245300474582
:100B700054202446245320485454502F312E310DF4
:100B80000A486F73743A2024460D0A416363657006
:100B9000743A20746578742F68746D6C0D0A436F15
:100BA0006E6E656374696F6E3A20636C6F73650D6A
:100BB0000A0D0A00E30004FA000100000001000031
:100BC0002100240027002A00000022002500280020
:100BD0002B00000020002300260029000202020250
:100BE00002020202040404040404040403030303D1
:100BF00003030303010101010101010101020408D2
:100C000010204080010204081020408001020408E6
:100C100010204080804020100804020100000001E4
:100C200002000000000000000403070600000000AE
:100C30000000000000000000000000003708432111
:100C4000AA2BBF3511241FBECFEFD0E1DEBFCDBF31
:100C500012E0A0E0B1E0EAEDF3E802C005900D92E9
:100C6000AA3BB107D9F71AE0AAEBB2E001C01D9286
:100C7000A038B107E1F71CE0C4E4DCE004C022972F
:100C8000FE010E94B041CC33D107C9F70E942E402B
:100C90000C94EB410C940000FC0188279927E89400
:100CA00021912032E9F3293010F02E30C8F32B3295
:100CB00041F02D3239F4689404C00E940507820F78
:100CC000911D219120532A30C0F31EF490958195F7
:100CD0009F4F0895FB01DC0102C005900D92415029
:100CE0005040D8F70895FB01DC0104C08D910190BC
:100CF000801921F441505040C8F7881B990B089582
:100D0000DC0101C06D9341505040E0F70895FB01B4
:100D1000DC0101900D920020E1F70895FB01DC0158
:100D20000D900020E9F711974150504028F00190B4
:100D300000200D92C9F708951C920895FB01DC0173
:100D40004150504030F08D910190801919F40020ED
:100D5000B9F7881B990B0895A0E0B0E0E2EBF6E04C
:100D60000C94BE417C01EB018A01690109C0CE01EE
:100D70002196F6010995F70181937F0101501040FA
:100D800001151105A1F7CDB7DEB7E8E00C94DA4103
:100D9000A0E0B0E0EEECF6E00C94BE41EC017B018B
:100DA0008A01690109C0CE012196F70161917F0195
:100DB000F60109950150104001151105A1F7CDB7B5
:100DC000DEB7E8E00C94DA41FB019F01E894423081
:100DD000C4F04532B4F44A3029F497FB1EF49095E0
:100DE00081959F4F642F77270E946541805D8A33EC
:100DF0000CF0895D8193CB010097A1F716F45DE2B9
:100E000051931082C9010C9432077AE0979F902D7C
:100E1000879F802D910D11240895FA01CF93FF93A0
:100E2000EF932230CCF02532BCF4C22F2C2F332785
:100E300044275527FF93EF930E948C41EF91FF9138
:100E4000605D6A330CF0695D6193B901CA0160505D
:100E500070408040904051F710828F919F91CF91C8
:100E60000C943207DC01FC01672F71917723E1F7C5
:100E7000329704C07C916D9370836291AE17BF0767
:100E8000C8F308959C01F999FECF32BD21BDF89AAF
:100E900080B508959C01F999FECF1FBA32BD21BDDE
:100EA00060BD0FB6F894FA9AF99A0FBE0895FC0146
:100EB000A681B7816D93B783A68381E090E0089502
:100EC000CF92DF92EF92FF920F931F93CF93DF9316
:100ED0007B018C010894E11CF11C011D111DC090C7
:100EE0002409442361F430912109369536953695CD
:100EF0003170AAE0B8E0CAE4D7E0DD2471C0909177
:100F000021099695969596959170CAE0D8E06AE485
:100F100077E0EC2DF0E0EE0FFF1FEE0FFF1FEC0F60
:100F2000FD1F25C0288139814A815B81211531054A
:100F300041055105C9F0DB01ED92FD920D931C9323
:100F40001397D801C701820F931FA41FB51F888371
:100F50009983AA83BB832091F1017C018D01E20E6C
:100F6000F11C011D111D91E024966C5F7F4FCE177F
:100F7000DF07C1F69170990F990F990F80912109A0
:100F8000877F892B37C04D915D916D917C9113972F
:100F9000411551056105710501F1ED2DE695E695C7
:100FA000E695F0E0EB5DF64F808190E02D2D277007
:100FB00002C0959587952A95E2F780FD0EC0E882DC
:100FC000F9820A831B834E0D5F1D601F711F4D93B5
:100FD0005D936D937C93139731E0D394149624968C
:100FE000DC1488F23170330F330F330F80912109F5
:100FF000877F832B80932109DF91CF911F910F91E0
:10100000FF90EF90DF90CF900895AAECB8E080E0D9
:1010100090E0FC01E65BF84F10821182128213828D
:10102000FC01E65FF74F10821182128213821D923B
:101030000496803C910569F7F999FECF86ED93E01F
:1010400092BD81BDF89A80B5809341071092420706
:1010500010924307109245071092440710924607DA
:10106000109247071092480710924907089510926E
:101070003C0710923B0788E692E090933A078093F2
:1010800039070895BF92CF92DF92EF92FF920F93AC
:101090001F93CF93DF932DB73EB72E5030400FB63E
:1010A000F8943EBF0FBE2DBFEDB7FEB7319609E3F2
:1010B00017E0ADB7BEB712961C930E9311978EE34F
:1010C00097E09383828389E990E09583848388ED18
:1010D00090E0978386838091230980871186809191
:1010E000F6018287138680911902848715860E94F3
:1010F0007931DD2490E7E92E93E0F92EEDB7FEB7C4
:101100003E960FB6F894FEBF0FBEEDBFB02EC12EB7
:101110000AE317E033C0F999FECFF2BCE1BCF89ABC
:1011200090B5F999FECF0894E11CF11CF2BCE1BC2A
:10113000F89A80B5D92FC0E000D000D000D0EDB72C
:10114000FEB73196ADB7BEB71196BC921197129605
:10115000CC92138302839E01280F311D3583248393
:101160000E947931D3940894E11CF11C8DB79EB78D
:1011700006960FB6F8949EBF0FBE8DBF80912409CE
:10118000D81608F4C8CF00D000D009E317E0ADB7F7
:10119000BEB712961C930E9311978CE297E01496AB
:1011A0009C938E9313970E947931EDB7FEB712830B
:1011B00001838DE097E0948383830E94793100D08E
:1011C000EDB7FEB73196ADB7BEB712961C930E932E
:1011D000119787EE96E09383828380E790E0958372
:1011E00084830E947931EDB7FEB736960FB6F89436
:1011F000FEBF0FBEEDBF81E0DF91CF911F910F9138
:10120000FF90EF90DF90CF90BF900895CF92DF9244
:10121000EF92FF920F931F93DF93CF9300D000D0F4
:10122000CDB7DEB70E943C3E7B018C016E01089475
:10123000C11CD11C0E9496370E942A2EC6016091C3
:101240005F010E942E2C8823E1F0E980FA800B8157
:101250001C8180EC98EDA4E5BCE7E80EF91E0A1F9E
:101260001B1F6091A10170E080E090E024E833E072
:1012700040E050E00E943A41E60EF71E081F191F99
:101280000EC00E943C3E6E197F09800B910B685E78
:1012900073408040904070F2EE24FF248701B70134
:1012A000C8010F900F900F900F90CF91DF911F9179
:1012B0000F91FF90EF90DF90CF9008951F9310E073
:1012C00060915F016F5F60935F018BE591E00E9429
:1012D0008C2D6AEF70E080E090E00E944A3E0E9410
:1012E00006099B01AC01611571058105910519F491
:1012F0001F5F153029F7B901CA011F910895CF93D7
:10130000DF939C0110920807FC01A081B181C0E02D
:10131000D0E00FC09C919D3231F09B3221F0892F9B
:1013200080538A3068F4FE01E85FF84F908321967D
:101330001196F901808191810A96A817B90750F397
:10134000C85FD84F18821196F901B183A08388E055
:1013500097E00E944C06DF91CF910895AF92BF9223
:10136000CF92DF92EF92FF920F931F93CF93DF9371
:101370008DB79EB708970FB6F8949EBF0FBE8DBF6E
:10138000EDB7FEB7319609E317E0ADB7BEB71296D9
:101390001C930E93119785E893E09383828389E9E8
:1013A00090E09583848388ED90E0978386830E9404
:1013B00079310F900F900F900F90EDB7FEB7128319
:1013C000018382E793E0948383830E9479313CE92F
:1013D000E32E31E0F32EDD24C0E0D0E00F900F903B
:1013E0000F900F90B02EC12E03E613E07C2FAD2E90
:1013F000D70114968C91149781FF3CC012964D91A1
:101400005C91139711966C9111978C91C43129F4CA
:10141000282F30E02C53304002C0282F30E0EDB7A9
:10142000FEB73C970FB6F894FEBF0FBEEDBF3196E6
:10143000ADB7BEB71196BC9211971296CC9213839A
:1014400002835583448380E090E0613011F481E0B1
:1014500090E097838683318720877287A3860E94D6
:101460007931D394EDB7FEB73C960FB6F894FEBF32
:101470000FBEEDBF219685E090E0E80EF91ECE315B
:10148000D10509F0B3CF28E0E22E27E0F22E80E567
:1014900090E0B7010E941121ADB7BEB718970FB603
:1014A000F894BEBF0FBEADBFEDB7FEB7319609E3EE
:1014B00017E012961C930E93119789E493E093839F
:1014C0008283D4821582F782E6820E9479310F905E
:1014D0000F900F900F90EDB7FEB7128301838EE34C
:1014E00093E0948383830E94793100D0EDB7FEB7F7
:1014F0003196ADB7BEB712961C930E93119783E148
:1015000093E09383828380E790E0958384830E94B5
:101510007931EDB7FEB736960FB6F894FEBF0FBE21
:10152000EDBF81E0DF91CF911F910F91FF90EF9080
:10153000DF90CF90BF90AF9008954F925F926F92DF
:101540007F928F929F92AF92BF92CF92DF92EF9253
:10155000FF920F931F93DF93CF930F92CDB7DEB718
:101560000E942D3B5B016C012DB73EB728503040E7
:101570000FB6F8943EBF0FBE2DBFEDB7FEB7319644
:1015800009E317E0ADB7BEB712961C930E931197FF
:1015900081E994E09383828389E990E09583848351
:1015A00088ED90E0978386830E94793100D0EDB773
:1015B000FEB73196ADB7BEB712961C930E93119736
:1015C00084E794E09383828388EC90E0958384831E
:1015D000A682B782C086D1860E9479310F900F9083
:1015E000EDB7FEB73196ADB7BEB712961C930E930A
:1015F00011978AE594E09383828380912309848301
:1016000015828091A101868317820E94793190E032
:10161000EDB7FEB738960FB6F894FEBF0FBEEDBF1C
:10162000780106E514E023C000D000D000D0EDB76B
:10163000FEB73196ADB7BEB71196EC9211971296E0
:10164000FC9213830283A92FB0E0AB5DB64F8C915F
:101650008483158299830E94793199819F5FEDB7C8
:10166000FEB736960FB6F894FEBF0FBEEDBF809161
:101670002309A9E36A2EA7E07A2E9817A8F200D0D2
:1016800000D0ADB7BEB712967C926E9211978AE4E5
:1016900094E014969C938E9313970E947931992429
:1016A0000F900F900F900F90C301762C892EF1E4CC
:1016B0004F2EF4E05F2E66C0A92DB0E0FD01E65389
:1016C000F74F60816623A9F1CD01880F991F880F1C
:1016D000991FFC01E65BF84FE080F18002811381E5
:1016E000FC01E65FF74FAE14BF04C006D10648F018
:1016F00020813181428153812A193B094C095D09BE
:1017000008C020813181428153812E193F09400B4D
:10171000510BAA0FBB1FAA0FBB1FA65FB74F8D911E
:101720009D910D90BC91A02D8E5F9F4FAF4FBF4FED
:1017300021F420E030E040E050E08DB79EB70A97FA
:101740000FB6F8949EBF0FBE8DBFEDB7FEB73196B2
:10175000ADB7BEB711967C92119712968C925382B8
:1017600042826483158226833783408751870E9493
:1017700079319394EDB7FEB73A960FB6F894FEBF61
:101780000FBEEDBF80912409981608F495CF48E06C
:10179000E42E47E0F42E80E590E0B7010E9411218D
:1017A0002DB73EB72A5130400FB6F8943EBF0FBE5A
:1017B0002DBFEDB7FEB7319609E317E0ADB7BEB761
:1017C00012961C930E9311978FEE93E0938382836E
:1017D00080912109817084831582809121098695E9
:1017E0008170868317828091210986958695817004
:1017F0008087118680912109829581708287138666
:101800008091310990913209A0913309B091340946
:1018100084879587A687B7878091F601808B118A88
:1018200080910502828B138A80910F02848B158A26
:1018300080911902868B178AF18EE08E0E94793191
:10184000EDB7FEB73C960FB6F894FEBF0FBEEDBFE6
:101850003196ADB7BEB712961C930E9311978DECCF
:1018600093E09383828380914207848315828091E1
:10187000430786831782809144079091450791879B
:1018800080878091460790914707A0914807B091C3
:10189000490782879387A487B5870E947931EDB77E
:1018A000FEB73A960FB6F894FEBF0FBEEDBF128397
:1018B00001838EEA93E0948383830E94793100D080
:1018C000EDB7FEB73196ADB7BEB712961C930E9327
:1018D00011978AE893E09383828380E790E0958371
:1018E00084830E947931EDB7FEB736960FB6F8942F
:1018F000FEBF0FBEEDBF81E00F90CF91DF911F9132
:101900000F91FF90EF90DF90CF90BF90AF909F909E
:101910008F907F906F905F904F900895CF93DF935B
:10192000FC01AC014B5F5F4F8581803221F4CA011D
:101930000E949D0A47C0C0E6D1E0A0E0B0E0682F59
:10194000772767FD7095E881F981849190E086178B
:10195000970709F040C03196249130E0FA01818167
:10196000992787FD909528173907A9F5AA0FBB1F5E
:10197000AA0FBB1FAE59BE4FED91FC91CA0109954C
:10198000882301F500D000D000D0EDB7FEB7319626
:1019900089E397E0ADB7BEB712969C938E931197EB
:1019A0008FE991E09383828383E091E09583848340
:1019B0000E947931EDB7FEB736960FB6F894FEBFA8
:1019C0000FBEEDBF62E370E080E090E00E944A3E0F
:1019D000DF91CF91089511962496AF30B10509F0AB
:1019E000B2CFF0CFBF92CF92DF92EF92FF920F93E0
:1019F0001F936C01FC01B080E1800E942D3B20E828
:101A000031E541E050E00E948C418B2D8F77280F0B
:101A1000311D411D511DFF2400E010E0CA01B90134
:101A2000A80197010E948C41F0E8BF22B62AF60176
:101A3000B0821F910F91FF90EF90DF90CF90BF90F9
:101A400008956F927F928F929F92AF92BF92CF92A2
:101A5000DF92EF92FF920F931F934C01FC01708075
:101A600061800E942D3BA62CBB24CC24DD242FE7D3
:101A7000E22EE720FF24E60CF11C0027F7FC00957E
:101A8000102F20E831E541E050E00E948C41CA016E
:101A9000B901A60195010E948C41E61AF70A080BCC
:101AA000190BC801B701A60195010E948C41F0E80D
:101AB0007F22762AF40170821F910F91FF90EF90A0
:101AC000DF90CF90BF90AF909F908F907F906F905E
:101AD0000895EF92FF921F93CF93DF93182F7B010E
:101AE0000E942D3B9B01AC01C12FD0E02F5F3F4FE7
:101AF0004F4F5F4FCE01880F991F880F991FFC0130
:101B0000E65BF84F2083318342835383FC01E65F19
:101B1000F74FE114F10449F48EEF9FEFAFEFBFEF01
:101B200080839183A283B3830DC0C701AA2797FD49
:101B3000A095BA2F280F391F4A1F5B1F20833183BE
:101B400042835383C653D74F83E68883809121090C
:101B5000886080932109DF91CF911F91FF90EF90D2
:101B600008958F929F92AF92BF92CF92DF92EF92A1
:101B7000FF920F931F93CF93DF938C010E5F1F4F44
:101B800020E030E006C0F901E95FF84F90830F5F75
:101B90001F4FE22FD8019C91892F80538A3028F45F
:101BA0002F5F3F4F2530310571F7F0E0E85FF84FC8
:101BB000108288E097E00E944C06EC0197FD00C17E
:101BC0008091240990E08C179D070CF4F9C0F8016E
:101BD00080818D3309F057C0209709F4F1C08091BE
:101BE000210984FFEDC02197C8010196218120338E
:101BF00079F40E942D3BEC2FF0E0EE0FFF1FEE0F6B
:101C0000FF1FE65FF74F608371838283938319C060
:101C1000213309F0D5C068E077E040E320E031E00F
:101C20000E94E234882319F460E070E007C088E085
:101C300097E00E944C06BC0197FDC2C08C2F0E9409
:101C4000690D00D000D000D0EDB7FEB7319689E322
:101C500097E0ADB7BEB712969C938E9311978BEA1F
:101C600091E09383828389E990E0958384830E9445
:101C7000793181E0EDB7FEB736960FB6F894FEBF26
:101C80000FBEEDBF9EC000D000D000D0EDB7FEB7B4
:101C9000319689E397E0ADB7BEB712969C938E93C9
:101CA000119788EA91E09383828389E990E0958394
:101CB00084830E947931EDB7FEB736960FB6F8945B
:101CC000FEBF0FBEEDBF209721F48091240990E064
:101CD00003C08C2F9C2F9150C0E0D0E0E92EFF2450
:101CE000082F10E039E3C32E37E0D32E22EA822EEC
:101CF00021E0922E95EAA92E91E0B92E58C090913C
:101D0000210990FF39C091FD37C0809105028823D9
:101D100011F092FD31C000D000D000D0ADB7BEB7F9
:101D20001196EDB7FEB7D282C1821396BC92AE92E5
:101D30001297F90183E0F595E7958A95E1F7EB5D58
:101D4000F64F808190E02770307002C0959587959E
:101D50002A95E2F78170907015969C938E93149754
:101D60000E9479312DB73EB72A5F3F4F0FB6F894E6
:101D70003EBF0FBE2DBF1AC000D000D000D0EDB7BF
:101D8000FEB73196ADB7BEB71296DC92CE921197E0
:101D900093828282158214820E947931EDB7FEB758
:101DA00036960FB6F894FEBF0FBEEDBF21969E018A
:101DB0002E0D3F1D201731070CF4A1CF81E001C08B
:101DC00080E0DF91CF911F910F91FF90EF90DF9016
:101DD000CF90BF90AF909F908F900895DF92EF9239
:101DE000FF920F931F93CF93DF9300D000D009E3AE
:101DF00017E0ADB7BEB712961C930E93119782EA07
:101E000098E014969C938E9313970E947931FF2447
:101E10000F900F900F900F90D02EE12E08E017E05A
:101E2000CCE9D8E021C08F2D68E077E00E94122035
:101E300000D000D000D0EDB7FEB73196ADB7BEB739
:101E40001196DC9211971296EC92D383C28315837C
:101E500004830E947931F394EDB7FEB736960FB63E
:101E6000F894FEBF0FBEEDBF80912409F816D8F29A
:101E700000D000D089E397E0ADB7BEB712969C932F
:101E80008E93119786E998E014969C938E931397FE
:101E90000E9479310F900F900F900F90DF91CF91AA
:101EA0001F910F91FF90EF90DF90089500D000D028
:101EB00000D0EDB7FEB7319689E397E0ADB7BEB776
:101EC00012969C938E93119783E198E0938382837B
:101ED00089E990E0958384830E9479318DB79EB71C
:101EE00006960FB6F8949EBF0FBE8DBF0E94EE0EF1
:101EF00081E00895CF92DF92FF920F931F93DF93BB
:101F0000CF930F92CDB7DEB72DB73EB72E503040EE
:101F10000FB6F8943EBF0FBE2DBFEDB7FEB731969A
:101F200009E317E0ADB7BEB712961C930E93119755
:101F300083E698E09383828389E990E095838483A4
:101F4000809123098683178280E190E091878087C2
:101F50008091F60182871386809119028487158605
:101F60000E947931EDB7FEB73E960FB6F894FEBFEA
:101F70000FBEEDBF0E94EE0E00D000D0ADB7BEB7D1
:101F800012961C930E93119787E598E014969C93F4
:101F90008E9313970E94793190E00F900F900F90DD
:101FA0000F90F02E012F53E5C52E58E0D52E23C0FB
:101FB00000D000D000D0EDB7FEB73196ADB7BEB7B8
:101FC0001196FC92119712960C93D382C282A92F7C
:101FD000B0E0A55DB64F8C918483158299830E94F1
:101FE000793199819F5FEDB7FEB736960FB6F894B9
:101FF000FEBF0FBEEDBF809123099817C8F200D035
:1020000000D000D0EDB7FEB7319689E397E0ADB7C9
:10201000BEB712969C938E9311978AE198E09383B2
:10202000828380E790E0958384830E947931EDB7C5
:10203000FEB736960FB6F894FEBF0FBEEDBF81E037
:102040000F90CF91DF911F910F91FF90DF90CF9074
:1020500008959C0180911902882311F081E0089570
:10206000C90168E077E040E322E031E00E94E23419
:10207000882331F088E097E00E942421811181E0DB
:1020800008956F927F928F929F92AF92BF92CF925C
:10209000DF92EF92FF920F931F93DF93CF93CDB711
:1020A000DEB7E5970FB6F894DEBF0FBECDBF73E085
:1020B000A72EB12CA80EB91EC5010E942910882395
:1020C00009F4EDC00CE911E0EE24CC24DD244E012E
:1020D0000894811C911C62E0662E712C6C0E7D1E92
:1020E0002C2D9D2DD80114968C91149781FF3BC007
:1020F00011968C911197813009F41C92D401ECE671
:10210000F2E085E001900D928150E1F7822FB3015A
:102110004AE050E00E94E406C50168E077E040E351
:1021200094010E94E2348823F1F0F801F180F1E09B
:10213000FF1619F4D801FC9216C088E097E00E94BF
:102140004C069C01B4E1CB1611F4245C3F4F37FDE3
:1021500008C08F2D90E0821793071CF0F8012083B0
:1021600002C0EE24E3940894C11CD11C0B5F1F4FE6
:10217000FEE1CF16D10409F0B3CFC50168E077E0E6
:1021800040E325E031E00E94E234882351F088E00A
:1021900097E00E942E3580E590E068E077E00E94AD
:1021A000EC20EE2089F000D000D000D0EDB7FEB7D3
:1021B000319689E397E0ADB7BEB712969C938E93A4
:1021C00011978EE792E090C00E94C820C50168E098
:1021D00077E040E329E031E00E94E2348823A1F176
:1021E0008E010A5F1F4FC501B80140E32DE031E0C9
:1021F0000E94E234882309F467C088E097E0B801C0
:1022000040E150E00E949E06009709F05DC080E426
:1022100090E068E077E00E94EC202DB73EB72850B0
:1022200030400FB6F8943EBF0FBE2DBFEDB7FEB7DE
:10223000319689E397E0ADB7BEB712969C938E9323
:10224000119786E592E016C02DB73EB72850304072
:102250000FB6F8943EBF0FBE2DBFEDB7FEB7319657
:1022600089E397E0ADB7BEB712969C938E93119712
:102270008CED91E09383828389E990E09583848358
:1022800083E591E0978386830E94793181E0EDB701
:10229000FEB738960FB6F894FEBF0FBEEDBFE596B9
:1022A0000FB6F894DEBF0FBECDBFCF91DF911F9167
:1022B0000F91FF90EF90DF90CF90BF90AF909F90E5
:1022C0008F907F906F90089500D000D000D0EDB730
:1022D000FEB7319689E397E0ADB7BEB712969C93EF
:1022E0008E93119788E092E09383828389E990E04E
:1022F000958384830E94793181E0EDB7FEB73696ED
:10230000C9CF8F929F92AF92BF92CF92DF92FF92EE
:102310000F931F93DF93CF9300D000D0CDB7DEB7DC
:10232000A3E0CA2ED12CC80ED91EC6010E942910C6
:10233000882309F483C083E789831A821B821C8265
:1023400010E0F2E08F2E912C8C0E9D1E5E01089401
:10235000A11CB11C1AC0812F90E0B4014AE050E0EA
:102360000E94E406C60168E077E040E395010E9420
:10237000E234882349F088E097E00E942E35812FCF
:1023800068E077E00E9437201F5F809124091817CA
:1023900010F38DE68983FF24E2E08E2E912C8C0EC3
:1023A0009D1E5E010894A11CB11C1AC00F2D10E0E7
:1023B000C801B4014AE050E00E94E406C60168E0AA
:1023C00077E040E395010E94E234882341F088E001
:1023D00097E00E944C06055D164FD8018C93F3944C
:1023E00080912309F81610F30E946120EDB7FEB723
:1023F00038970FB6F894FEBF0FBEEDBF319689E354
:1024000097E0ADB7BEB712969C938E9311978EEE60
:1024100097E09383828389E990E09583848383E5C1
:1024200091E0978386830E94793181E0EDB7FEB712
:1024300038960FB6F894FEBF0FBEEDBF0F900F9009
:102440000F900F90CF91DF911F910F91FF90DF9030
:10245000CF90BF90AF909F908F9008958F929F9252
:10246000AF92BF92CF92DF92EF92FF920F931F93A2
:10247000CF93DF93EC017A018B01CB01BA010E946B
:102480001A3A4C01C801B7010E94143A5C018889CC
:10249000882309F481C0D880D7FE21C0C98021E0FB
:1024A0002C15E8F4C801B70120E831E541E050E01F
:1024B0000E948C41CA01B9012C2D30E040E050E06F
:1024C0000E948C412FE7D2222D2D30E040E050E0D9
:1024D000621773078407950709F05EC031C0C80111
:1024E000B7010E94083A288130E090E0059667E045
:1024F00070E00E94794102C0359527958A95E2F7F0
:1025000020FF4AC0C801B7010E940E3AD82E888128
:1025100087FF16C08981882319F4D0FE11C03CC002
:10252000813071F48FE1D816B9F12DE1D21609F09E
:1025300042C0C801B7010E94023A0297E1F52CC0DF
:102540008CE390E0889E9001899E300D989E300D1E
:1025500011242A0D3B1D4A815B8124173507E0F0C9
:102560008C819D8182179307B8F0EE81FF813097AF
:1025700099F0241B350B40E0C901BF010E94654161
:102580006E9FC0016F9F900D7E9F900D112482174A
:10259000930719F441E001C040E0842FDF91CF910F
:1025A0001F910F91FF90EF90DF90CF90BF90AF9071
:1025B0009F908F900895D0FCC3CFEECF982F9B01B2
:1025C00080914107981768F461E1969FB00111244A
:1025D00068527C4FC90141E150E022E437E00E949B
:1025E000AC060895CF92DF92EF92FF920F931F9364
:1025F000DF93CF93CDB7DEB762970FB6F894DEBF07
:102600000FBECDBF8C010D5F1F4FC8010E942E353C
:10261000C80168E077E040E321E131E00E94E23464
:10262000882309F415C188E097E00E944C067C01DC
:102630002FEF8F3F92070CF40BC18091410790E080
:10264000E816F9060CF004C18DB79EB708970FB6CF
:10265000F8949EBF0FBE8DBFEDB7FEB7319609E36C
:1026600017E0ADB7BEB712961C930E93119781E891
:1026700096E09383828389E990E09583848388ED53
:1026800090E0978386830E94793100D0EDB7FEB742
:102690003196ADB7BEB712961C930E9311978AE58B
:1026A00096E0938382838091230984831582F78245
:1026B000E68280911902808711860E947931EDB7F8
:1026C000FEB73A960FB6F894FEBF0FBEEDBFFFEF10
:1026D000EF16FFEFFF0609F48FC08E2D7E010894E0
:1026E000E11CF11CB7010E94DE128A81823018F0D1
:1026F000C7010E94210D2DB73EB7225130400FB6C1
:10270000F8943EBF0FBE2DBFEDB7FEB7319609E37B
:1027100017E0ADB7BEB712961C930E9311978BE3DB
:1027200096E0938382838989848315828981868355
:1027300017828A81808711868B819C81938782870B
:102740008D819E81958784878F81988597878687DD
:1027500089859A85918B808B0E94793190E0EDB7C5
:10276000FEB772960FB6F894FEBF0FBEEDBF6801BC
:10277000B7E3EB2EB6E0FB2E8E01055F1F4F22C0A4
:1027800000D000D000D0EDB7FEB73196ADB7BEB7E0
:102790001196CC9211971296DC92F382E282D801C4
:1027A000A90FB11D8C91848315829A8B0E94793177
:1027B0009A899F5FEDB7FEB736960FB6F894FEBFC5
:1027C0000FBEEDBF809123099817D0F200D000D042
:1027D00089E397E0ADB7BEB712969C938E9311979D
:1027E00084E396E014969C938E9313970E9479311C
:1027F0000F900F900F900F9000D000D009E317E0DA
:10280000EDB7FEB7128301838BE096E09483838358
:102810000E94793100D0EDB7FEB73196ADB7BEB7A3
:1028200012961C930E93119784EE95E09383828306
:1028300080E790E0958384830E94793181E0EDB751
:10284000FEB736960FB6F894FEBF0FBEEDBF01C0BF
:1028500080E062960FB6F894DEBF0FBECDBFCF9179
:10286000DF911F910F91FF90EF90DF90CF9008952F
:102870002F923F925F926F927F928F929F92AF9230
:10288000BF92CF92DF92EF92FF920F931F93DF934D
:10289000CF93CDB7DEB761970FB6F894DEBF0FBE0A
:1028A000CDBFD82EE82EFF2487E090E0E80EF91E79
:1028B0004E010894811C911C89E3A82E87E0B82E54
:1028C0000BE0202E312C2C0E3D1EC5015A2CC92E9A
:1028D0001AEC612E17E0712E73C08D2DB4010E9489
:1028E000DE128A81823018F0C4010E94210DADB73A
:1028F000BEB754970FB6F894BEBF0FBEADBFEDB7CD
:10290000FEB731961296BC92AE92119781ED97E088
:1029100093838283158304838989868317828981BF
:10292000808711868A81828713868B819C81958717
:1029300084878D819E81978786878F819885918BEB
:10294000808B89859A85938B828B0E94793110E0E8
:10295000ADB7BEB754961CC000D000D000D0EDB7C4
:10296000FEB73196ADB7BEB71296BC92AE92119734
:102970008DEC97E093838283D101A10FB11D8C91DF
:10298000848315820E9479311F5FADB7BEB716965A
:102990000FB6F894BEBF0FBEADBF809123091817C4
:1029A000D8F200D000D0EDB7FEB75182C282748257
:1029B00063820E947931D3940F900F900F900F9003
:1029C0000D2D10E0E016F1062CF080914107D8168D
:1029D00008F483CF61960FB6F894DEBF0FBECDBF6B
:1029E000CF91DF911F910F91FF90EF90DF90CF90EB
:1029F000BF90AF909F908F907F906F905F903F902F
:102A00002F900895FF920F931F93CF93DF938DB76D
:102A10009EB70C970FB6F8949EBF0FBE8DBFEDB753
:102A2000FEB73196C9E3D7E0ADB7BEB71296DC93D7
:102A3000CE93119788E997E0938382838091410731
:102A400084831582809123098683178280911902DD
:102A5000808711868EE390E0938782870E94793188
:102A6000EDB7FEB73C960FB6F894FEBF0FBEEDBFB4
:102A700080E00E94381400D000D0ADB7BEB71296E7
:102A8000DC93CE9311978DE897E014969C938E93E8
:102A900013970E9479310F900F900F900F908091B3
:102AA0004107893080F111E0CE01FC2E092FCEE6DE
:102AB000D7E01CC000D000D000D0EDB7FEB73196F3
:102AC000ADB7BEB71196FC92119712960C93D383B3
:102AD000C283358324830E9479311F5FEDB7FEB72F
:102AE00036960FB6F894FEBF0FBEEDBF212F30E033
:102AF0008091410790E0019768E070E00E94794181
:102B000062177307BCF6DF91CF911F910F91FF9071
:102B100008952F923F924F925F926F927F928F9281
:102B20009F92AF92BF92CF92DF92EF92FF920F935C
:102B30001F93DF93CF9300D0CDB7DEB78C010D5F2D
:102B40001F4FC8010E942E350E942D3B5B016C0176
:102B50000E94F9392C01C601B5010E94023A3C01DC
:102B6000C601B5010E940E3A4C01C601B5010E9492
:102B70001A3A9A838983C601B5010E94143A1C014E
:102B8000C80168E077E040E325E131E00E94E234EB
:102B9000882361F088E097E00E944C064C01009782
:102BA00029F4C601B5010E940E3A4C01C80168E043
:102BB00077E040E327E131E00E94E234882329F006
:102BC00088E097E00E944C063C01C80168E077E08D
:102BD00040E329E131E00E94E234882329F088E0D3
:102BE00097E00E944C062C012DB73EB72C51304087
:102BF0000FB6F8943EBF0FBE2DBF0DB71EB70F5FC7
:102C00001F4F39E3E32E37E0F32EADB7BEB7129670
:102C1000FC92EE92119788E595E0F8019383828308
:102C200089E990E0958384838091EC018683178203
:102C30008091F6018087118680910F02828713862A
:102C40008091F101848715868091FB018687178624
:102C500080910002808B118AC601B50120E831E520
:102C600041E050E00E948C41D80153963C932E9352
:102C700052978CE390E0E981FA819C01E29FC001C8
:102C8000E39F900DF29F900D1124820D931D559698
:102C90009C938E93549757969C928E9256975996E2
:102CA0007C926E9258975B965C924E925A970E94D5
:102CB00079314DB75EB7485E5F4F0FB6F8945EBF8F
:102CC0000FBE4DBFADB7BEB71296FC92EE921197F4
:102CD0008CE495E014969C938E9313970E9479311F
:102CE00000E00F900F900F900F90BE2CEF2C28E477
:102CF000C22E25E0D22E21C000D000D000D0EDB7EA
:102D0000FEB73196ADB7BEB71196BC921197129629
:102D1000EC92D382C282A02FB0E0A55DB64F8C9119
:102D2000848315820E9479310F5FEDB7FEB7369626
:102D30000FB6F894FEBF0FBEEDBF8091230999E353
:102D4000892E97E0992E0817B8F200D000D0ADB7C1
:102D5000BEB712969C928E92119784E495E01496D9
:102D60009C938E9313970E9479310F900F900F9040
:102D70000F900E94021500D000D0EDB7FEB79282EE
:102D8000818285E295E0948383830E94793100D02B
:102D9000EDB7FEB73196ADB7BEB712969C928E9244
:102DA00011978DEF94E09383828380E790E0958381
:102DB00084830E947931EDB7FEB736960FB6F8944A
:102DC000FEBF0FBEEDBF81E00F900F90CF91DF915E
:102DD0001F910F91FF90EF90DF90CF90BF90AF9039
:102DE0009F908F907F906F905F904F903F902F902B
:102DF00008950F931F938DB79EB708970FB6F89459
:102E00009EBF0FBE8DBFEDB7FEB7319609E317E049
:102E1000ADB7BEB712961C930E9311978DEC96E04A
:102E20009383828389E990E09583848388ED90E0A1
:102E3000978386830E947931EDB7FEB738960FB637
:102E4000F894FEBF0FBEEDBF0E94021500D000D067
:102E5000ADB7BEB712961C930E9311978EEA96E00B
:102E600014969C938E9313970E94793100D0EDB7FE
:102E7000FEB73196ADB7BEB712961C930E9311975D
:102E800086E896E09383828380E790E0958384834D
:102E90000E947931EDB7FEB736960FB6F894FEBFB3
:102EA0000FBEEDBF81E01F910F9108950F931F9307
:102EB0008C0102960E942E35D80112960C91112792
:102EC00007FD10950053104043E0000F111F4A9575
:102ED000E1F700D000D000D0EDB7FEB7319689E31E
:102EE00097E0ADB7BEB712969C938E93119787EC7F
:102EF00097E09383828389E990E0958384830E949D
:102F00007931EDB7FEB736960FB6F894FEBF0FBE17
:102F1000EDBF802F0E94381481E01F910F9108951A
:102F2000DF92EF92FF920F931F93DF93CF93CDB772
:102F3000DEB761970FB6F894DEBF0FBECDBF20910C
:102F40004107821708F043C0222309F440C090E0F3
:102F500001968C0164E0000F111F6A95E1F7080FDC
:102F6000191F08521C4F51E1D52E7E010894E11C17
:102F7000F11C13C0C701B80141E150E022E437E081
:102F80000E94AC06C8014197B70141E150E02AE434
:102F900037E00E94C8060F5E1F4F209141072D9D0C
:102FA000C001112488529C4F0817190718F32150AB
:102FB00020934107F999FECF1FBA86ED93E092BDA9
:102FC00081BD20BD0FB6F894FA9AF99A0FBE6196AA
:102FD0000FB6F894DEBF0FBECDBFCF91DF911F912A
:102FE0000F91FF90EF90DF900895CF93DF93EC0166
:102FF0002396CE010E942E35CE010E9429108823EF
:1030000009F450C0CE0168E077E040E321E131E00F
:103010000E94E234882309F445C088E097E00E94CA
:103020004C069C018FEF2F3F380781F41092410727
:10303000F999FECF1FBA86ED93E092BD81BD10BC19
:103040000FB6F894FA9AF99A0FBE09C08091410719
:1030500090E02817390734F5822F0E94901700D08E
:1030600000D000D0EDB7FEB7319689E397E0ADB759
:10307000BEB712969C938E93119789EB95E093833C
:10308000828389E990E0958384830E94793181E08D
:103090002DB73EB72A5F3F4F0FB6F8943EBF0FBE25
:1030A0002DBF01C080E0DF91CF910895982F8091CE
:1030B0004107981760F481E1989FC001112488525C
:1030C0009C4F41E150E02AE437E00E94C806089591
:1030D000BC01909141079E33F0F481E1989FC001BB
:1030E000112488529C4F41E150E02AE437E00E94CD
:1030F000C806209141072F5F20934107F999FECF21
:103100001FBA86ED93E092BD81BD20BD0FB6F89445
:10311000FA9AF99A0FBE0895BF92CF92DF92EF927A
:10312000FF920F931F93DF93CF93CDB7DEB76397D3
:103130000FB6F894DEBF0FBECDBF7C018C010D5FD2
:103140001F4FC8010E942E35C8010E9429108823F4
:1031500009F403C1C80168E077E040E321E131E010
:103160000E94E234882309F4F8C088E097E00E94C6
:103170004C066C012FEF8F3F92070CF4EEC080914C
:10318000410790E0C816D9060CF0E7C01A830983FE
:1031900087E690E0E80EF91E0DC0C8016BE171E012
:1031A00043E050E00E949E06009779F00F5F1F4FAA
:1031B0001A83098309811A81D8018C91882309F423
:1031C000CCC00E151F0548F3C8C00D5F1F4F1A83F2
:1031D00009838E010F5F1F4FC8010E947F098B8BEF
:1031E000C8010E947F098B83C8010E947F098C83DC
:1031F000C8010E947F099E838D83C8010E947F09B8
:1032000098878F83C8010E947F099A878987C801A0
:103210000E947F099C878B87FF24B02EE12E8E01B0
:10322000035F1F4F09C08B2D9E2D0E947F09F8015F
:10323000EF0DF11D8083F39480912309F81698F324
:1032400006C0FC01EF0DF11D1082F39402C0CE0107
:103250000D96B5E0BF15A8F78C81823020F0CE0125
:1032600003960E94F20C00D000D000D0EDB7FEB75C
:10327000319609E317E0ADB7BEB712961C930E93D3
:10328000119782EF94E09383828389E990E095839C
:1032900084830E947931EDB7FEB736960FB6F89465
:1032A000FEBF0FBEEDBFBE016D5F7F4FFFEFCF16BC
:1032B000FFEFDF06C1F4CB010E94681800D000D0F8
:1032C000ADB7BEB712961C930E93119785ED94E09F
:1032D00014969C938E9313970E9479310F900F90C0
:1032E0000F900F9022C08C2D0E94561800D000D055
:1032F00000D0EDB7FEB73196ADB7BEB712961C93AE
:103300000E93119787EB94E0938382830894C11CFA
:10331000D11CD582C4820E947931EDB7FEB73696B2
:103320000FB6F894FEBF0FBEEDBF00D000D089E30A
:1033300097E0ADB7BEB712969C938E93119786E92E
:1033400094E014969C938E9313970E94793181E0B8
:103350000F900F900F900F9001C080E063960FB612
:10336000F894DEBF0FBECDBFCF91DF911F910F91BB
:10337000FF90EF90DF90CF90BF9008950E949C2027
:103380000E94B724AAECB8E080E090E0FC01E65B84
:10339000F84F1082118212821382FC01E65FF74F10
:1033A00010821182128213821D920496803C910534
:1033B00069F708950F931F93CF93DF93EC01239642
:1033C000CE010E942910882309F4E7C0CE0168E0ED
:1033D00077E040E32FE131E00E94E234882311F0EE
:1033E0000E94BE19CE0168E077E040E323E231E0BD
:1033F0000E94E234882309F44AC088E097E00E94E2
:103400004C06181619060CF042C02DB73EB72850CE
:1034100030400FB6F8943EBF0FBE2DBFEDB7FEB7DC
:10342000319609E317E0ADB7BEB712961C930E9321
:10343000119781EE92E09383828389E990E09583EE
:1034400084838AE090E0978386830E9479310F908D
:103450000F900F900F90EDB7FEB71283018384EDAC
:1034600092E0948383830E9479310F900F900F90A4
:103470000F9080913F079091400720913D07309138
:103480003E07821B930B0E944A2D0E940C20CE0106
:1034900068E077E040E327E231E00E94E2348823ED
:1034A00099F080910807813339F48091210980FDDA
:1034B0000BC00E94412508C0803331F4809121095E
:1034C00080FF02C00E943725CE0168E077E040E32C
:1034D0002AE231E00E94E2348823D9F08091080783
:1034E000813351F48091210984FD13C00E94BE19DB
:1034F0008091210980610BC0803359F480912109AA
:1035000084FF07C00E94BE19809121098F7E80939D
:103510002109CE0168E077E040E32DE231E00E942E
:10352000E234882371F088E097E00E944C06181678
:1035300019061CF40E94082504C0892B71F50E940D
:1035400000252DB73EB7285030400FB6F8943EBF47
:103550000FBE2DBFEDB7FEB7319689E397E0ADB74B
:10356000BEB712969C938E93119787EC92E093834B
:10357000828389E990E09583848383E591E0978352
:1035800086830E94793181E0EDB7FEB738960FB699
:10359000F894FEBF0FBEEDBF01C080E0DF91CF9178
:1035A0001F910F910895BF92CF92DF92EF92FF92F9
:1035B0000F931F93DF93CF9300D0CDB7DEB77C017D
:1035C0008C010D5F1F4FC8010E942E35C8010E945B
:1035D0002910882309F4A0C01A83098327E630E064
:1035E000E20EF31E0DC0C80160E371E043E050E05D
:1035F0000E949E06009779F00F5F1F4F1A83098380
:1036000009811A81D8018C91882309F485C00E158F
:103610001F0548F381C00D5F1F4F1A8309830E9465
:10362000BE19FF2400E713E0EE246E010894C11CCC
:10363000D11CEEEFBE2E37C0C6010E947F09F9995A
:10364000FECF1FBA12BD01BD90BD0FB6F894FA9A15
:10365000F99A0FBEF999FECF1FBA0F5F1F4F12BD27
:1036600001BD0150104080BD0FB6F894FA9AF99A46
:103670000FBE0097A9F02F2D30E0F901EE0FFF1FCC
:10368000EE0FFF1FE65FF74FA0E0B0E0808391836D
:10369000A283B3832653374FF901B082EE24E3941B
:1036A000F3940E5F1F4F80912409F81608F4C4CFDD
:1036B000EE2031F00E942D3B4091EC010E9460070A
:1036C0002DB73EB7285030400FB6F8943EBF0FBE1E
:1036D0002DBFEDB7FEB7319689E397E0ADB7BEB722
:1036E00012969C938E9311978AED96E09383828332
:1036F00089E990E09583848383E591E097838683CD
:103700000E94793181E0EDB7FEB738960FB6F89494
:10371000FEBF0FBEEDBF01C080E00F900F90CF91B4
:10372000DF911F910F91FF90EF90DF90CF90BF90AE
:103730000895EF92FF920F931F939B01AC0180912C
:10374000FA089091FB08A091FC08B091FD08009741
:10375000A105B10549F42093FA083093FB08409382
:10376000FC085093FD0854C079018A01E81AF90A4F
:103770000A0B1B0BD801C701CD97A105B10508F4B1
:1037800047C02093FA083093FB084093FC085093FD
:10379000FD0889E799E00E94DD2D0E943C3E7B01F7
:1037A0008C010E9496370E942A2E89E799E00E9498
:1037B000FC30882361F40E943C3E6E197F09800B27
:1037C000910B683C71058105910558F319C08091F2
:1037D00022098F70809322098091220982958F702F
:1037E00090E00397ACF08091E201882389F060912A
:1037F000BA027091BB0285E591E00E94E62708C0FD
:1038000080912209982F907F905F8F70892BE2CF53
:103810001F910F91FF90EF900895EF92FF920F93F9
:103820001F939B01AC018091A6018823C9F180916F
:10383000220982958F70A1F58091FE089091FF0872
:10384000A0910009B09101090097A105B10569F0A7
:1038500079018A01E81AF90A0A0B1B0BD801C70182
:1038600081589145A140B040D8F02093FE08309394
:10387000FF0840930009509301090E945E097B01F3
:103880008C01611571058105910551F00E94003B85
:103890008091210985FF04C0C801B7010E94612BF6
:1038A0001F910F91FF90EF9008950E941F270E9493
:1038B0009D250E9405089091DD0180E02091D801AE
:1038C000820F911D9093BB028093BA026CE370E06B
:1038D00080E090E00E94F73A8091210985FD03C0C5
:1038E00080E090E002C08AE89BE20E94A03B64EF87
:1038F00071E080E090E00E944A3E80E00E94D52680
:103900008BEA98E061E00E9428226091BA027091EF
:10391000BB0285E591E00E94E627882321F0809193
:1039200022098F7004C0809122098F70806180937A
:10393000220964EF71E080E090E00E944A3E0E941C
:10394000B7240E942D3B0E940D1C80E00E94D526CA
:10395000089582E00E949921282F30E086FF41C01F
:103960002F7030702230310591F02430310509F18B
:1039700021303105B1F587FF03C00E94412508952C
:10398000609144027091450281E799E009C087FF88
:1039900003C00E943725089589E799E060E070E050
:1039A0000E946F2460ED77E080E090E00E944A3E44
:1039B000089587FF06C081E00E9499210E940C2093
:1039C000089520912209822F8F7090E06091230941
:1039D000019670E00E9479418F70207F282B209300
:1039E000220908952F923F924F925F926F927F9299
:1039F0008F929F92AF92BF92CF92DF92EF92FF92FF
:103A00000F931F93DF93CF93CDB7DEB7A9970FB670
:103A1000F894DEBF0FBECDBF2091EC012C8B30910E
:103A2000F6013B8B0E9496370E942A2E9C019093B0
:103A30000309809302090097F9F010923C07109255
:103A40003B0782EF92E090933E0780933D0790936F
:103A5000400780933F07C90184549D4F0E948E0CFC
:103A600080913F079091400720913D0730913E079C
:103A7000821B930B0E944A2D0E94A91C0E942D3B81
:103A80004B015C018091080990910909A0910A09F4
:103A9000B0910B0988159905AA05BB0509F4A3C2C5
:103AA0008092080990920909A0920A09B0920B0924
:103AB00080E00E94D5268091210981FF0FC080916E
:103AC000310990913209A0913309B09134098816D7
:103AD0009906AA06BB0610F00E9400250E94E2216A
:103AE0008091210984FDC4C083FF04C04C89442314
:103AF00009F0BEC0C501B4012CE330E040E050E065
:103B00000E948C4179018A018091040990910509F4
:103B1000A0910609B0910709E816F9060A071B07E4
:103B200009F4A6C0E0920409F09205090093060981
:103B30001093070910E066249B89892F90E099A7CC
:103B400088A78AC0862DBE016F5F7F4F0E94DE125C
:103B5000CE010196B501A4010E942E12882309F41A
:103B60007AC029853A852115310509F474C0A091E0
:103B70002309AE8B77241A8A190144245524B62DC3
:103B8000BF5FBFA353C08A898C0DE82EFF24C701F5
:103B90000196E8A5F9A5E817F907E1F1ABA1BCA1E9
:103BA0008C9190E00C2C02C0959587950A94E2F7D1
:103BB00080FD30C0EDA1FEA1808190E00C2C02C000
:103BC000959587950A94E2F780FF24C08701000F3E
:103BD000111F000F111F065F174F60910F0270E059
:103BE00080E090E0A20191010E943A4124E630E099
:103BF00040E050E00E948C41D8012D933D934D93BD
:103C00005C931397EAECF8E0EE0EFF1EEFA1D701EC
:103C1000EC9311E00894C11CD11CF8E0CF16D1043C
:103C200009F0B1CF73942A89285F2A8B3E897316D5
:103C300090F4872D90E0CC24DD24AC014B5D564FF1
:103C40005CA34BA3ABE0B0E0AC0FBD1FA80FB91F46
:103C5000BEA3ADA398CF639480914107681608F482
:103C600071CF112329F0C501B4014C890E9460076E
:103C70008091210983FF4BC13324FB89EF2FF0E0B2
:103C8000FC8FEB8F2B882A94222D30E0C901880FFE
:103C9000991F880F991FAC01465B584F5E8F4D8F5F
:103CA000DC01A65FB74FB8A3AF8FF901E653F74F1A
:103CB000FAA3E9A30FC1832D90E0FC01EB5DF64F61
:103CC0002081F32DFF0FFF0FFF0FFD8B662477245C
:103CD000422F50E0588F4F8BDC01A55DB64FBA8F55
:103CE000A98FFD88F60C8F89988D062C02C09595BA
:103CF00087950A94E2F7CF2CDD2480FF53C086011C
:103D0000000F111F000F111FF801E65FF74F8081B0
:103D10009181A281B38188169906AA06BB0608F490
:103D2000D0C08F2D60E00E947820C6010196EB8DF7
:103D3000FC8DE817F907E1F0F0924207F601E6532F
:103D4000F74F808180934307065B184FD8018D9110
:103D50009C91F401E81BF90BF0934507E0934407AD
:103D60008092460790924707A0924807B092490771
:103D7000F601EE0FFF1FEE0FFF1FDF01A65BB84F2E
:103D80001D921D921D921C921397E65FF74F1082B1
:103D90001182128213822AEC38E0C20ED31ED601A1
:103DA0001C928FC09601220F331F220F331F8901EF
:103DB000065B184FF80180819181A281B38188163A
:103DC0009906AA06BB0608F47CC0AAE04A2EA8E021
:103DD0005A2E420E531EF20180819181A281B3813D
:103DE00088169906AA06BB0608F06BC08F2D61E005
:103DF0000E947820FB89FF2309F463C0C601019665
:103E00002B8D3C8D2817390709F45BC0A98DBA8D1D
:103E10008C9190E0062C02C0959587950A94E2F764
:103E200080FF4FC0BC89BB2309F44BC0809121099E
:103E300084FD47C08091FB01F801208131814281DE
:103E40005381280F311D411D511DAD8DBE8D2D9308
:103E50003D934D935C93139780910002E82EFF24CD
:103E600000E010E084EC9FEFAFEFBFEFE80EF91E2B
:103E70000A1F1B1FF20180819181A281B381E80E8C
:103E8000F91E0A1F1B1FAF8DB8A1ED92FD920D9375
:103E90001C931397EAECF8E0CE0EDF1ED6018C914E
:103EA000E9A1FAA1808382169306A406B50648F01C
:103EB0008E149F04A006B10620F4822D61E00E94BA
:103EC00078200894611C711CF8E06F16710409F0E9
:103ED00008CF339480912309381608F4ECCE0E9461
:103EE000B72430912409EAE0F8E020E00DC0819188
:103EF0009191A191B1910197A109B1098E5F9F4F55
:103F0000AF4FBF4F20F02F5F231788F361C05B894D
:103F1000552369F08091210984FF09C0109124097B
:103F200040E021E030E08B89682F70E02EC09C8952
:103F30009923A1F331C0842F90E06217730711F128
:103F4000DC01F3E0B695A795FA95E1F7542F577089
:103F5000FD01EB5DF64F808190E0052E02C0959546
:103F600087950A94E2F780FF0DC0A55DB64F8C914E
:103F700090E002C0959587955A95E2F780FF02C0C0
:103F800061E006C04F5F2F5F3F4F4117A0F260E036
:103F90008B8981500E9478200E94B724C501B4010A
:103FA00023E030E040E050E00E948C419B01AC01F6
:103FB0002F583D4F81E0D9016C910E94F623C50135
:103FC000B4010E94991BC501B4010E940D1C0BC0D5
:103FD0000E949C2080912109877F80932109B091C4
:103FE000F601BB8B94CFA9960FB6F894DEBF0FBE37
:103FF000CDBFCF91DF911F910F91FF90EF90DF9098
:10400000CF90BF90AF909F908F907F906F905F9078
:104010004F903F902F900895E0913509F091360927
:1040200009950895DB01482F50E0495F5F4F84E018
:10403000440F551F8A95E1F750961C92509720E047
:1040400030E0F999FECFC901840F951F92BD81BD63
:10405000F89A80B5FD01E20FF31F8083882331F0C9
:104060002F30310519F02F5F3F4FEBCF0895DB0163
:10407000482F50E0495F5F4F94E0440F551F9A95D9
:10408000E1F750961C92509720E030E0FD01E20FDE
:10409000F31FE081F999FECF1FBAC901840F951F64
:1040A00092BD81BDE0BD0FB6F894FA9AF99A0FBEA1
:1040B000EE2331F02F30310519F02F5F3F4FE6CF5F
:1040C000089580ED93E0FC01E55AFA4FE081F999FB
:1040D000FECF1FBA92BD81BDE0BD0FB6F894FA9A2B
:1040E000F99A0FBE019623E0863D920761F7089585
:1040F000282F277086958695869590E0662369F02F
:10410000FC01EB5DF64F81E090E002C0880F991F43
:104110002A95E2F72081282B0DC0FC01EB5DF64FBC
:1041200081E090E002C0880F991F2A95E2F7809500
:1041300020812823208308951092250910922609B2
:1041400010922709109228091092290910922A0921
:104150000895ECE9F1E020E030E0F999FECF32BDBE
:1041600021BDF89A80B580832F5F3F4F35962E3161
:10417000310599F78091E7018F5F8093230990E0E3
:1041800023E0880F991F2A95E1F780932409089569
:10419000EDE2F2E08DE190E02081F999FECF1FBAC7
:1041A00092BD81BD20BD0FB6F894FA9AF99A0FBE60
:1041B000019735972FEF8F3F920771F78091E701B5
:1041C0008F5F8093230990E033E0880F991F3A9521
:1041D000E1F7809324090895AC01FB010FC0F99920
:1041E000FECF1FBADA01A80FB11DB2BDA1BD20BD1F
:1041F0000FB6F894FA9AF99A0FBE31968E2F861B55
:104200002081222361F7F999FECF1FBA480F511D73
:1042100052BD41BD10BC0FB6F894FA9AF99A0FBE80
:104220000895AC01FB018E2F861BF999FECF9A01F0
:10423000280F311D32BD21BDF89A80B580838823B7
:1042400011F03196F0CF0895582F282F392FF9010A
:104250008E2F851BF999FECF90E0805C9F4F92BD19
:1042600081BDF89A80B59081882331F0992349F077
:10427000891739F43196ECCF80E0992319F481E065
:10428000089580E00895CF92EF920F938CE099E02B
:1042900063E142E124E105E176E1E72E57E1C52E35
:1042A0000E94322A0F91EF90CF900895EF92FF92E3
:1042B0000F931F93CF93DF93E82E162F042FF22E28
:1042C000662321F0623081F4222371F08E2D0E944A
:1042D000DB3F892B11F000E024C0FF2011F480E0C7
:1042E00001C080E8082B1DC0C0E0D0E08E2D0E94E8
:1042F000DB3F892B81F4113031F0123061F483E01F
:10430000C032D80744F461E070E080E090E00E94A1
:104310004A3E2196EBCFFF2019F4C052D3400CF057
:104320000068802FDF91CF911F910F91FF90EF9048
:1043300008950F931F93082F10913709107861E0AB
:1043400070E080E090E00E944A3E8FE10E94DB3FF7
:10435000892B21F48FE1602F41E013C08EE10E9490
:10436000DB3F892B21F48EE1602F42E00AC08DE112
:104370000E94DB3F892B11F040E007C08DE1602FE8
:1043800044E0212F0E945621482F8091370990E068
:104390008F709070242F30E0892B39F42F7030709B
:1043A000232B71F0842F806406C02F703070232B74
:1043B00039F4842F8062409337091F910F9108953B
:1043C000842FF9CF8BE00E94DB3F40E020910A026E
:1043D00030E08217930709F041E0440F440F8091C9
:1043E00021098B7F842B809321090895EF92FF92FE
:1043F0000F931F938C01ECE0EE2EE9E0FE2E6AE0B5
:1044000070E00E947941C7014AE050E00E942741D4
:10441000C8016AE070E00E947941BC01C7014AE02E
:1044200050E00E9427411F910F91FF90EF90089557
:10443000CF93DF93EC0104C08CE099E00E946740C9
:10444000FE01219664916623B9F7DF91CF9108951B
:104450000F931F93CF93DF938C01462F8CE099E04D
:1044600060E00E944529E80104C08CE099E00E94C8
:1044700067409E01201B822FFE01219664916623D6
:10448000A1F7992787FD9095C0E1D0E0C81BD90B13
:1044900005C080E89AE00E9418222197D7FFF9CF43
:1044A000DF91CF911F910F910895EF92FF920F939B
:1044B0001F93CF93DF937C018C01000F111F000F1E
:1044C000111F0E0D1F1D04561E4FF801828193818E
:1044D00060E00E9428228DE49AE061E00E94282298
:1044E0008CE099E060E041E00E944529F801848178
:1044F00080FF05C08CE099E00E94292904C08CE06F
:1045000099E00E943329F3E1EF16F10409F45EC04B
:1045100084E1E816F10454F4E1E0EE16F104B1F0A0
:10452000FCE0EF16F10409F08CC065C08BE1E816E1
:10453000F10409F46AC0ECE1EE16F10409F475C067
:10454000F4E1EF16F10409F07CC047C08091A101AD
:10455000C82FD0E0E097D7FD05C08BE49AE00E9419
:10456000182207C089E49AE00E941822D095C195CC
:10457000DF4FCE0164E070E00E9479418CE099E069
:104580004AE050E00E94274187E49AE00E94182206
:10459000CE0164E070E00E947941BC01B4E0660F96
:1045A000771FBA95E1F7681B790B29F484E49AE048
:1045B0000E94182206C08CE099E04AE050E00E9478
:1045C00027418FE39AE00E94182260C08DE39AE0B1
:1045D0000E9418226091FB0120C0809100028C3360
:1045E00020F08BE39AE00E9418226091000270E0B4
:1045F0006C53704007C07091DD0160E08091D8017C
:10460000680F711D8CE099E00BC0609123028DE072
:1046100070E00E94E83E609123028CE099E070E037
:104620004AE050E00E94274131C0809128026FEF9C
:1046300070E0681B71098CE00E94E83E60912802DE
:10464000ECCFF701EE0FFF1FEE0FFF1FEE0DFF1D6A
:10465000E456FE4F81816081813051F4662319F464
:1046600084E39AE002C087E39AE00E94182207C020
:104670008CE099E070E04AE050E00E94274187E139
:10468000E816F10419F482E39AE00EC0C7014397DB
:10469000029740F0E8E1EE16F10421F0F1E1EF16A7
:1046A000F10421F48DE29AE00E941822DF91CF916B
:1046B0001F910F91FF90EF900895EF92FF920F934B
:1046C0001F93182F092F0E945522212F302FC90127
:1046D0008C013AEAE32E82E00E949921482F282F8C
:1046E00030E0C9018F70907082309105D1F0843034
:1046F000910551F1019709F066C0F801EE0FFF1F17
:10470000EE0FFF1FE00FF11FE456FE4F848180FF84
:104710005DC090818181891709F458C09F5F9083A3
:1047200055C0F801EE0FFF1FEE0FFF1FE00FF11F46
:10473000E456FE4F848180FF46C08081882309F4BF
:1047400042C0815080833FC046FF3DC047FF0BC041
:1047500080912D02882311F0E0922D020E94C82042
:10476000FF24F39434C00330110541F48091AB0170
:10477000882309F1FF240CE010E029C00C3011055A
:1047800021F4FF240EE010E022C00531110541F4B0
:1047900080910502882379F4FF2407E110E017C017
:1047A0000231110541F48091F601882321F4FF24A0
:1047B00005E110E00CC0C80101966EE170E00E94B6
:1047C00079418C0103C0442309F485CFFF24C8013B
:1047D0000E945522FF2009F47ECF8CE099E00E94D0
:1047E00033291F910F91FF90EF9008950F931F931E
:1047F000CF93DF93482F062F8CE099E060E00E9472
:104800004529809122098F7019F48FE69AE010C033
:104810008DE69AE00E941822609122096F708CE068
:1048200099E070E04AE050E00E9427418BE69AE070
:104830000E9418228091210980FD03C08FE59AE033
:104840000AC081FD06C082FF0AC08091050288234C
:1048500031F083E59AE061E00E94282226C0E091D1
:104860002209EF70F0E0EB5DF64F1081C1E0D0E07F
:10487000809122098F7051F48091F60190E0C81761
:10488000D90721F410FD06C06DE405C010FD02C07B
:104890006FE501C0602F8CE099E00E94674021968F
:1048A000C930D10511F01695E3CF8EE49AE00E944D
:1048B00018228CE099E06FE041E00E94452960E019
:1048C0008091220982958F7009F061E08CE099E077
:1048D0000E94F728DF91CF911F910F910895EF92D9
:1048E000FF920F931F93CF93DF938C017B018CE09A
:1048F00099E00E9474298CE099E060E040E00E9419
:104900004529C0E0D0E0F801EC0FFD1F60818CE08C
:1049100099E070E04AE050E00E94274185E79AE084
:104920000E9418222196C330D10569F7F8016381EE
:104930008CE099E070E04AE050E00E9427418CE072
:1049400099E060E041E00E94452983E79AE00E94F7
:1049500018228CE099E0B7014AE050E00E9427411C
:10496000DF91CF911F910F91FF90EF900895EF92FB
:10497000FF920F931F93CF93DF9383E060E00E9439
:10498000873F0AE219E09091210990FF0BC091FD49
:1049900009C080910502882311F092FD03C0F8013F
:1049A000608101C060E0C7E0D0E0E62EFF2486E130
:1049B00060E00E94873FB7010C2E02C07595679595
:1049C0000A94E2F7617085E10E94873F86E161E029
:1049D0000E94873F2197FFEFCF3FDF0741F701504C
:1049E000104089E00432180771F683E061E00E940C
:1049F000873FDF91CF911F910F91FF90EF90089526
:104A0000809121098D7F809321090E94B724089508
:104A1000DF92EF92FF920F931F93D82E882309F114
:104A20000E942D3B7B018C016D2D70E080E090E0B9
:104A300020E13EE040E050E00E943A41E60EF71EE1
:104A4000081F191FE0923109F092320900933309CF
:104A500010933409809121098260809321090E947A
:104A6000B7241F910F91FF90EF90DF9008958091F0
:104A700021098E7F809321090E94B7240E94C820BB
:104A80000895809121098160809321090E94B724B3
:104A90000E94C8200895AF92BF92CF92DF92FF92FA
:104AA0000F931F93CF93DF935B016C01FF24C1E051
:104AB000D0E03CC08CE099E00E9474298CE099E041
:104AC00060E040E00E9445290F2D10E0B8016F5FC3
:104AD0007F4F8CE099E04AE050E00E94274110921D
:104AE0002509109226091092270910922809109280
:104AF000290910922A0943E0169507954A95E1F78E
:104B00000B5D164F8F2D87709E0102C0220F331F41
:104B10008A95E2F7C901F8012081282B20830E94A1
:104B2000B724C601B5010E944A3EF394809124093E
:104B3000F81608F4BFCFFF24FBCF64EF71E080E0EC
:104B400090E00E944A3EF999FECF12BC11BCF89A3F
:104B500090B5943620F48AE0989F902D1124983CCB
:104B600059F4F999FECF8DE190E092BD81BDF89A9C
:104B700080B58A3A09F089C00E94C82080E490E09C
:104B800064E371E00E94EC2080E590E06DE371E069
:104B90000E94EC2082EC9AE060E00E94282283EBE5
:104BA0009AE061E00E94282280E790E0F999FECF28
:104BB0001FBA92BD81BD10BC0FB6F894FA9AF99A4B
:104BC0000FBE019628E08030920781F720E730E0A1
:104BD000E1E0F0E043E5F999FECF1FBA32BD21BD17
:104BE00040BD0FB6F894FA9AF99A0FBEF999FECF24
:104BF0001FBA2F5F3F4F32BD21BD21503040CF0142
:104C00006AE070E00E947941605D60BD0FB6F89483
:104C1000FA9AF99A0FBEF999FECF1FBA2E5F3F4F4D
:104C200032BD21BDCF016AE070E00E947941805D14
:104C300080BD0FB6F894FA9AF99A0FBE225F3F4FE3
:104C400083E02037380711F03196C5CF80ED93E02F
:104C50002FEFF999FECF1FBA92BD81BD20BD0FB6CF
:104C6000F894FA9AF99A0FBE019633E0863D9307BD
:104C700081F764EF71E080E090E00E944A3EE091AD
:104C80003509F0913609099514C00E94A92020ED3C
:104C900033E0F999FECF32BD21BDF89A80B5F90114
:104CA000E55AFA4F80832F5F3F4F83E0263D380758
:104CB00081F780E00E94992190E08F70907082309F
:104CC000910521F18430910521F1019709F04CC043
:104CD00064E670E080E090E00E944A3E8DE10E9430
:104CE000DB3F892B29F460E273E080E090E00BC0A9
:104CF0006091140270E080E090E028EE33E040E044
:104D000050E00E943A410E944B252EC08DE190E078
:104D100020C083EA9AE060E00E94282260ED77E0FC
:104D200080E090E00E944A3E82E99AE060E00E94C2
:104D3000282282E89AE061E00E94282280E00E9416
:104D4000992186FFFBCF8CE099E00E94742980E0D6
:104D500090E00E945D2380912D02882329F0E0914C
:104D60003509F091360909958CE061E00E94483FD1
:104D70008DE061E00E94483F609123028DE070E089
:104D80000E94E83E809128026FEF70E0681B710975
:104D90008CE00E94E83E08950E94B73B90E00596A3
:104DA00067E070E00E9479410895DF92EF92FF92F0
:104DB0000F931F93D82E0E942D3B7B018C018CE01A
:104DC00099E060E04D2D0E944529C801B7010E947D
:104DD0001A3A0E94F6218EE79AE00E941822C80132
:104DE000B7010E94143A0E94F6218BE79AE00E94D4
:104DF00018220E94CC26E82FF0E0EE0FFF1FEE5C99
:104E0000FD4F808191810E94182289E79AE00E94DB
:104E10001822C801B7010E94023A0E94F62187E7D2
:104E20009AE00E941822C801B7010E940E3A0E941F
:104E3000F6211F910F91FF90EF90DF9008950F934F
:104E40001F93DF93CF93CDB7DEB728970FB6F894B3
:104E5000DEBF0FBECDBF83E061E00E94483F81E02E
:104E600061E00E94483F86E161E00E94483F85E1A1
:104E700061E00E94483F83E061E00E94873F81E05B
:104E800061E00E94873F1092250910922609109236
:104E90002709109228091092290910922A090E94C4
:104EA000B72481E060E00E94873F11E01093810009
:104EB0008CE061E00E94483F8DE061E00E94483F45
:104EC000609123028DE070E00E94E83E809128020C
:104ED0006FEF70E0681B71098CE00E94E83E8CE087
:104EE00099E060E142E020E00E947C298BE060E0F4
:104EF0000E94483F8BE061E00E94873F8EED99E081
:104F00000E945736809121098160817C809321091C
:104F1000109222091093230988E0809324091092AB
:104F20003109109232091092330910923409DE01CE
:104F30001196E4E7F2E001900D928150E1F78CE0E8
:104F400099E061E08E010F5F1F4FA8010E940129C7
:104F50001A821B8281E08C838CE099E060E0A801DA
:104F60000E9401298CE161E00E94483F8CE160E0F1
:104F70000E94873F8FE160E00E94483F8EE160E041
:104F80000E94483F8DE160E00E94483F8FE161E070
:104F90000E94873F8EE161E00E94873F8DE161E0E2
:104FA0000E94873F0E94CD2A882329F480912109FD
:104FB00080628093210928960FB6F894DEBF0FBE59
:104FC000CDBFCF91DF911F910F9108950F931F9344
:104FD000DF93CF93CDB7DEB728970FB6F894DEBF37
:104FE0000FBECDBFFC018B0180911E0285838CE436
:104FF00094E0BF0144E00E943831882311F490E02E
:1050000034C010934502009344028091AB01882381
:1050100029F087E491E00E94D33421C08091B0014F
:1050200089838091B5018A838091BA018B838091B5
:10503000BF018C838091C4018D838091C9018E83CF
:105040008091CE018F838091D3018887CE01019614
:10505000BE016B5F7F4F40E050E00E94173190E04F
:10506000882309F491E081E09827892F28960FB6CC
:10507000F894DEBF0FBECDBFCF91DF911F910F918E
:1050800008950F931F938C01FC01868160E00E94BC
:10509000873F81E090E00E94A33EF801868161E0B5
:1050A0000E94873F81E090E00E94A33EF801868144
:1050B00060E00E94873F84E690E00E94A33E1F913B
:1050C0000F910895CF92DF92EF92FF920F931F936B
:1050D000CF93DF93D82EC92E282F392FC9018C01E9
:1050E000C0E0D0E0E62EFF24F801878161E00E9455
:1050F000483FB7010C2E02C0759567950A94E2F7F8
:105100006170F80187810E94873F21960F5F1F4FD2
:10511000C830D10549F78D2D9C2D0E944128DF9183
:10512000CF911F910F91FF90EF90DF90CF90089556
:10513000CF92DF92EF92FF920F931F93CF93DF9363
:10514000D82EC92E282F392FC9018C01C0E0D0E0FC
:10515000E62EFF24F801878161E00E94483FB701F5
:105160000C2E02C0759567950A94E2F76170F801FC
:1051700087810E94873F21960F5F1F4FC430D10562
:1051800049F78D2D9C2D0E944128DF91CF911F91D1
:105190000F91FF90EF90DF90CF9008951F93CF93E2
:1051A000DF93EC01162F8C81642F0E94873F8D8145
:1051B0008F3F19F060E00E94873F8F8584FF05C014
:1051C000CE01612F0E9462280EC0612F70E084E042
:1051D000759567958A95E1F7CE010E949828CE01D2
:1051E000612F0E949828DF91CF911F91089541E08F
:1051F0000E94CE2881E090E0089540E00E94CE28F1
:105200000895EF92FF920F931F93CF93DF938C013A
:105210007A016770660F660F660F60640E94FD2852
:10522000C0E0D0E0D801ED91FC91D701AC0FBD1FDB
:105230000190F081E02DC8016C9109952196C8304C
:10524000D10581F7DF91CF911F910F91FF90EF90E2
:105250000895FC016089862F8160808B6960CF0191
:105260000E94FD280895FC0160896E7F608B686054
:105270000E94FD280895FC016089862F8460808B40
:105280006C60CF010E94FD280895DF93CF93CDB7C6
:10529000DEB728970FB6F894DEBF0FBECDBF9C01D6
:1052A000FE013196A4E8B2E088E00D9001928150B1
:1052B000E1F7F9018389481710F0482F4150E42F96
:1052C000F0E0EE0FFF1FEC0FFD1F8181680F60689B
:1052D000C9010E94FD2828960FB6F894DEBF0FBEC4
:1052E000CDBFCF91DF91089561E00E94FD2880ED50
:1052F00097E00E94A33E0895CF93DF93EC014230E4
:1053000018F08F8588608F874B8B1C8A222329F0A9
:10531000413019F48F8584608F8780E593EC0E947B
:10532000A33E8C8160E00E94873F8E8160E00E94F6
:10533000873F8D818F3F19F060E00E94873F6F8526
:1053400064FD1DC0CE0163E00E94982884E991E1CC
:105350000E94A33ECE0163E00E94982884E991E177
:105360000E94A33ECE0163E00E94982886E990E067
:105370000E94A33ECE0162E00E94982816C060629F
:10538000CE010E94FD2884E991E10E94A33E6F8531
:105390006062CE010E94FD2886E990E00E94A33E53
:1053A0006F856062CE010E94FD286F856062CE012C
:1053B0000E94FD2884E0888BCE010E943B29CE010B
:1053C0000E94742982E0898BCE0166E00E94FD284C
:1053D000DF91CF9108956F927F928F92AF92CF928B
:1053E000EF920F931F93DF93CF93CDB7DEB73C01BE
:1053F000162F842FF301448325830683E782C0861A
:10540000A18682869D8593879E8594879F859587B3
:105410009889968761E00E94483FF30185818F3F1C
:1054200019F061E00E94483FF301868161E00E942B
:10543000483F112319F0F301178603C080E1F301FF
:105440008787C30160E141E020E00E947C29CF9181
:10545000DF911F910F91EF90CF90AF908F907F9041
:105460006F9008958F92AF92CF92EF920F931F9308
:10547000CF93DF93DC01362F542F722F102FAE2CD9
:105480008C2C13961C921E92129780E892E0119633
:105490009C938E9300D000D0EDB7FEB73196CDB778
:1054A000DEB71982118212821382CD0161E0432F8F
:1054B0002FEF052FE72EC12E0E94EB290F900F90A2
:1054C0000F900F90DF91CF911F910F91EF90CF90A0
:1054D000AF908F900895482F6AE00E945941282F7D
:1054E00030E084E0220F331F8A95E1F7842F0E9479
:1054F0005941892F820F0895EF92FF920F931F93C6
:105500007C010EED19E0C80168E670E00E94853567
:10551000C80160E00E940736F70180810E946B2A73
:10552000682FC8010E940736F70181810E946B2A0B
:10553000682FC8010E940736F70182810E946B2AFA
:10554000682FC8010E940736F70183810E946B2AE9
:10555000682FC8010E940736F70184810E946B2AD8
:10556000682FC8010E940736F70185810E946B2AC7
:10557000682FC8010E940736F70186818E510E946C
:105580006B2A682FC8010E940736C8010E9437366F
:105590001F910F91FF90EF9008950F931F930EEDC1
:1055A00019E0C80168E670E00E948535C80160E036
:1055B0000E940736C8010E9437361F910F91089547
:1055C000DF92EF92FF920F931F937C010EED19E093
:1055D000C80168E670E00E948535C80160E00E945D
:1055E0000736C8010E943736C80168E670E047E018
:1055F00050E00E945436C8010E949835282F2F771A
:1056000022952F709AE0D92E2D9D900111248F7034
:10561000820FF7018083C8010E949835282F2295B8
:105620002F702D9D900111248F70820FF7018183BF
:10563000C8010E949835282F2F7322952F702D9D19
:10564000900111248F70820FF7018283C8010E949C
:105650009835282F22952F702D9D900111248F7041
:10566000820FF7018383C8010E949835282F229565
:105670002F702D9D900111248F70820FF70184836C
:10568000C8010E949835282F22952F702D9D9001DA
:1056900011248F70820FF7018583C8010E9498350D
:1056A000282F2F70225E82958F708D9DC00111244E
:1056B000280FF70126831F910F91FF90EF90DF9045
:1056C00008950F931F93DF93CF93CDB7DEB727973E
:1056D0000FB6F894DEBF0FBECDBF8E010F5F1F4F18
:1056E000A8010E94D138898180688983C8010E94FD
:1056F0007C2A89818F778983C8010E947C2A27961A
:105700000FB6F894DEBF0FBECDBFCF91DF911F91D2
:105710000F9108950F931F93DF93CF93CDB7DEB70B
:1057200027970FB6F894DEBF0FBECDBF8E010F5F77
:105730001F4FC8010E94E02AC8010E94203A279604
:105740000FB6F894DEBF0FBECDBFCF91DF911F9192
:105750000F9108958EED99E00E9457360895DF92DB
:10576000EF92FF920F931F93CF93DF93D82E862F44
:10577000BA01213041F4675F7F4F9B0140E050E068
:10578000695070400EC0223029F020E030E040E047
:1057900050E007C0625070409B0140E050E06E5FF7
:1057A0007F4FE82EFF248CEB92E0E80EF91E8B0170
:1057B000E7010FC0F881E0E0898190E08E2B9F2BFC
:1057C000A0E0B0E0280F391F4A1F5B1F229602504D
:1057D00010400230110570F7CB018E7FD701A80F62
:1057E000B91F6817790779F08C9190E0A0E0B0E0DC
:1057F000BA2FA92F982F882702C040E050E0280F29
:10580000391F4A1F5B1FCA01AA27BB270097A105A2
:10581000B10599F7C90180959095ED2DF0E0E4541C
:10582000FD4F90838183DF91CF911F910F91FF9066
:10583000EF90DF9008951092D4021092D50280E488
:105840008093D0021092D1028093D20288E16EE060
:1058500044E150E020E00E94AF2B0895282F6623FA
:1058600021F08091E1028617E1F48091E202882321
:10587000C1F48091E3028833A1F48091DF028B3779
:1058800081F4E22FF92F80910E03838380910F031F
:10589000828380911003818380911103808381E052
:1058A000089580E008950F931F93BC010CEB12E064
:1058B000C8010E947135C80106966BE679E00E9426
:1058C00071351F910F910895EF92FF920F931F93DF
:1058D0007B010E94532C0AED12E0C801B7010E941F
:1058E0007935C801049761E779E00E9479351F9105
:1058F0000F91FF90EF900895CF92DF92EF92FF9279
:105900000F931F936C018B017A0185E499E00E944B
:10591000642CF8018081807F803E31F48CEB92E032
:105920006CE872E00E94713588E08093C8021092A2
:10593000C9028AEC92E06BED7AE049E050E00E9407
:105940006A061092CC0281E18093D302F092E002C9
:10595000E092E102D092DE02C092DF021092E202F7
:105960001092E4021092E5021F910F91FF90EF90C8
:10597000DF90CF900895EF92FF920F931F9302EC68
:1059800012E0C8010E94532C74E1E72EF12CE00EC6
:10599000F11EC8014896B7010E947935C70161E739
:1059A00079E00E9479350E941B2C1F910F91FF9086
:1059B000EF900895BC0181E08093380989E799E070
:1059C0000E94793508950F931F938C0188969093C8
:1059D000CC028093CD020E941B2C1092EE021092FA
:1059E000EF02045E1F4F82E36AE1A80122E00E94F9
:1059F000AF2BC8014A960E943D371F910F91089521
:105A0000CF93DF939C01862F80618093EB026430FB
:105A100029F02115310511F421E030E09091E002E8
:105A20008091DE028093E0029093DE029091E10289
:105A30008091DF028093E1029093DF02C5EED2E015
:105A40008881A901480F511D2C814C832883252F63
:105A50003327219752E0C13ED50791F71D861E8658
:105A600080E589871092CC0288E28093CD020E9463
:105A7000BB2C84E08B871C8682E36AE14CE150E01A
:105A800022E00E94AF2B86E390E00E943D37DF9139
:105A9000CF9108950F931F938C01809143099091AA
:105AA000440960E00E94002D89E18093EB02C80167
:105AB0000E94E32C1F910F9108950F931F93DF9382
:105AC000CF930F92CDB7DEB78C01045E1F4F1093BA
:105AD000CC020C511040802F845E8093CD028983CC
:105AE0000E941B2C085F1F4F1093E2028981845192
:105AF0008093E302085F1F4F88E26AE1A80121E07A
:105B00000E94AF2BC8014A960E943D370F90CF915B
:105B1000DF911F910F910895FF920F931F939C01A6
:105B2000F62E85E499E0B9010E94642C08EC12E09D
:105B300088E08093C8021092C902C80102966BEDFA
:105B40007AE049E050E00E946A068CE48093CD023E
:105B500081E18093D3020E941B2C1092E0028BE71C
:105B60008093E1028AE08093DE02F092DF021092DD
:105B7000E20288E38093E3021092E4021092E502CD
:105B8000025E1F4F80E3F80111928A95E9F7C80180
:105B900064EB7BE04AE050E00E946A0688E26AE13A
:105BA00040E450E021E00E94AF2B8AE590E00E94A3
:105BB0003D371F910F91FF900895EF92FF920F9341
:105BC0001F93BC0185E499E00E94642C08EC12E06C
:105BD000F8E0FF2EF092C8021092C902C8010296A6
:105BE0006BED7AE049E050E00E946A0684E580931C
:105BF000CD02EE24E394E092D3020E941B2CF0929B
:105C0000DE021092DF021092E0021092E10285E0C3
:105C10008093E202809174098093E3021092E4027F
:105C2000E092E502C8014E9662E470E048E350E07D
:105C30000E94800684E262E240E450E020E00E949C
:105C4000AF2B82E690E00E943D371F910F91FF90AD
:105C5000EF900895DF92EF92FF920F931F93CF93EF
:105C6000DF937C01009709F0B6C0809138098570F8
:105C7000F1F18091400290914102892BC1F50E947F
:105C800022378823A1F18CE892E00E94532C88E00F
:105C90008093C802E6E0FE2EF092C9028AEC92E000
:105CA00063ED7AE048E050E00E946A060CED12E0F5
:105CB000D8011D92FA94E9F7C8010A976BE679E0DA
:105CC0000E947135C801069669E779E00E9479352E
:105CD000C801049761E779E00E947935809138091D
:105CE0008860809338098AE290E00E943D37809175
:105CF00040029091410201969093410280934002AC
:105D000080913909813009F066C28091380981FF9C
:105D100062C202E000933909809142028F5F809352
:105D200042028F7110913A091295110F107E182BB3
:105D3000E0903B09D0903C0985E499E065E879E082
:105D40000E94642C78E0F72EF092C8021092C902EB
:105D50008AEC92E06BED7AE049E050E00E946A063E
:105D60008CE28093CD0286E08093D3020E941B2CAC
:105D7000E092E002D092E1028BE08093DE02109389
:105D8000DF02E2EEF2E0DF011D92FA94E9F7809182
:105D900043028093E4028D5F8093430280E6809308
:105DA000EA020093EB0283E08093EC021092ED0292
:105DB0001092EE021092EF021092F0021092F10295
:105DC0000093F20284E08093F3020093F40286E2EF
:105DD0008093F502B9C18932910508F4FCC1109194
:105DE000C802183009F002C28091C902863009F059
:105DF000FDC182EE92E061E779E044E050E00E946C
:105E00007306009709F0F2C18091D102813029F523
:105E100082EC92E00E94532C1092D00282E0809398
:105E2000D1028CED92E062ED72E00E94713582ED5C
:105E300092E06BE679E00E94713582EE92E068EDC7
:105E400072E00E94793588ED92E061E779E00E9486
:105E500079358AE290E00E943D378091380983FFCE
:105E6000BAC11091D102123009F0B5C188ED92E0AB
:105E700069E779E044E050E00E947306009709F07A
:105E8000AAC185E499E062ED72E00E947135109339
:105E90003809A1C1183009F09EC18091C902882338
:105EA00009F099C18091CA02853409F094C18AED44
:105EB00092E061E779E044E050E00E9473060097C9
:105EC00009F089C19091D302913009F58091DE02E9
:105ED0008830E9F4E0913D09F0913E09309719F0DE
:105EE00086ED92E009950E94BB2C1092DE02809113
:105EF000E002883F28F08091E1028F5F8093E10209
:105F00008091E002885F8093E002C70126C1E6E34A
:105F1000EE16F10418F4963009F05DC12091E0020C
:105F20002B3009F0BBC086ED92E065E879E044E0F3
:105F300050E00E947306009709F04DC18091EB027A
:105F4000382F82FF13C0E0913F09F091400930974C
:105F500009F49AC08091E10282958695877063E08A
:105F600040E050E020E030E009958EC09091CC02F6
:105F700080E02091CD02022F10E0082B192B809198
:105F8000EA02482F50E064E0559547956A95E1F79D
:105F9000CA01880F991F880F991F081B190B0451FC
:105FA000104017FF02C000E010E0E80180913909BD
:105FB000823079F531FF21C034FF1FC080E090E0CE
:105FC00060E00E94002D88E18093EB02E09141099E
:105FD000F0914209309719F420E030E007C0809139
:105FE000DF0282958695877009959C0183E08093F6
:105FF0003909C9010E94E32CEEC081E08093390980
:1060000034FF03C080E090E002C0C801019664E064
:10601000E0C0833059F50115110541F1E0913F09C8
:10602000F0914009309711F1440F551F440F551F4F
:10603000C70108974E5D5F4F8417950708F4AC01C0
:10604000C801840F951FE816F90610F0980103C0E7
:106050009701241B350B8091E1028295869587700C
:1060600060E00995882311F0C8010BC080913909BF
:10607000853009F4B0C08091EB0280FF09C0C801EF
:10608000019669E00E94002D85E080933909A3C044
:106090000115110509F4A1C0C8019AC0409144023C
:1060A00030E08091450290E02817390709F093C04D
:1060B0008091E102841709F08EC08091EB02682F75
:1060C00081FF4EC01092CC028CE28093CD020E94E0
:1060D000BB2C82E18093EB029091E0028091DE0282
:1060E0008093E0029093DE029091E1028091DF02C2
:1060F0008093E1029093DF02E5EEF2E021E030E0F0
:106100008081A901480F511D44831082252F332718
:10611000319752E0E13EF50799F715861686118210
:10612000128280914302838314828D5F80934302A5
:1061300082E0818B84E0828B95E0938B148A80E6E9
:106140008187938788E7848782E36AE140E250E0B1
:1061500022E00E94AF2B8AE390E00E943D373BC0D3
:1061600084FF39C09091CC0280E02091CD0230E0D4
:10617000282B392B8091EA02482F50E014E05595E6
:1061800047951A95E1F7CA01880F991F880F991F43
:10619000281B390B2451304037FF02C020E030E08B
:1061A0003093440920934309232B71F0EA01CC0F6B
:1061B000DD1FCC0FDD1FA29688EF9FEFE80EF91EC2
:1061C000EC16FD0640F009C060FF05C080E090E0DD
:1061D00060E00E94002DC0E0D0E0CE01DF91CF91C1
:1061E0001F910F91FF90EF90DF9008959AE2E916CA
:1061F000F10408F04FCEEFCFBC018091D302813083
:10620000A1F48091DE02882381F48091E602823439
:1062100061F486ED92E044E050E00E9473069C0138
:1062200080E0232B19F481E0089580E008950F9316
:106230001F93CF93DF939C01EB018A01009729F014
:1062400081E799E0B9010E947935209719F0CE01D4
:106250000E94DA2C0115110529F081E899E0B801B6
:106260000E94793581E0DF91CF911F910F910895C0
:10627000AF92BF92CF92DF92FF920F931F93CF9373
:10628000DF938C01EB01F42E38E341E050E060E055
:1062900070E018C0832F90E0FC01B3E0F595E7951E
:1062A000BA95E1F7E55BF64F877090705A016B0184
:1062B00004C0AA0CBB1CCC1CDD1C8A95D2F7208123
:1062C0002A292083315031F78BE699E0BE010E94E4
:1062D0007135C8016BE679E04F2D0E942E38DF91B1
:1062E000CF911F910F91FF90DF90CF90BF90AF9013
:1062F0000895CF92DF92EF92FF920F931F93DF9357
:10630000CF93CDB7DEB7EB84FC84CD84DE84DE0191
:106310001F9601C0D801F6018491882309F493C027
:106320000894C11CD11C843209F070C0F601089495
:10633000C11CD11C84918634B9F1873434F484347F
:1063400051F0853409F062C046C08C3489F0833541
:1063500009F05CC01EC08D010E5F1F4FF701668102
:1063600077818D919C914AE050E00E94E40659C0EB
:106370008D010C5F1F4F6D917D918D919C91D70187
:1063800016964D915C9117972AE030E00E940D0718
:1063900048C08D010E5F1F4F6D917C91F701868182
:1063A00097810E9487063DC08D010E5F1F4F6D9142
:1063B0007C910AC0D7011696ED91FC9117978193B5
:1063C0001796FC93EE931697FB016F5F7F4F8491B6
:1063D000882381F79FCF8D010E5F1F4F6D917C91B8
:1063E0000AC0D7011696ED91FC91179781931796E5
:1063F000FC93EE931697F999FECF72BD61BDF89AA2
:1064000080B56F5F7F4F882361F784CFF7012681C6
:106410003781F90181939F01F701378326838D012D
:1064200079CFD70116968D919C911797FC01019019
:106430000020E9F73197E81BF90B8E0F9F1FF7013A
:106440009783868367CFCF91DF911F910F91FF9044
:10645000EF90DF90CF9008958B9708F454C080910F
:10646000DF02833409F04FC08091E602823009F0E8
:106470004AC02091EA023091EB024091EC02509127
:10648000ED0280918A0990918B09A0918C09B091BD
:106490008D09281739074A075B07A9F59091CC02A7
:1064A00080E02091CD02AC01420F511D9A012C5089
:1064B0003140E6EDF3E01EC04533B9F4828185300A
:1064C00031F0863081F08230F1F482E008958091DD
:1064D0008909833031F08330B0F08550823098F4F0
:1064E00014C083E0089581E00895818190E00196D1
:1064F000E80FF91F40814F3F31F0CF01865D934097
:1065000082179307C8F280E0089584E008950F93FE
:106510001F93CF93DF93082F162F0E9422378823D3
:1065200009F4EFC0CCEBD2E08AE191E0FE019C01DE
:10653000119221503040E1F784E490E061E779E086
:1065400043E450E00E947C2CCE0106966BE679E095
:106550000E947135CE0168E972E00E94713582E8CF
:106560008093CD0281E18093D302112329F0CE01E3
:106570004E9668E972E004C0CE014E966DE779E070
:106580000E94793581E08093E6028093E70286E0FD
:106590008093E8021092E90280918A0990918B0918
:1065A000A0918C09B0918D098093EA029093EB023F
:1065B000A093EC02B093ED021092EF021092EE0263
:1065C000112319F480E090E002C080E890E09093FD
:1065D000F1028093F00282E093E06BE679E00E94A2
:1065E0007135A2EDB3E0ECE5F2E002C081918D934C
:1065F00032E0E036F307D1F785E38093D60391E0EC
:106600009093D7030093D8038DE38093D90387E059
:106610008093DA039093DB03ACEDB3E0EBE6F9E0B3
:1066200002C081918D9389E0E137F807D1F78CE0C2
:106630008093E20383EE93E0909397098093960909
:10664000A6E4B2E0FD0101900020E9F73197EA1BD2
:10665000FB0BE093E303EC012196F0E09F012A0F8E
:106660003B1F02C08D918993A217B307D9F7DF01B1
:10667000AC51BC4FB0939709A0939609033049F5EC
:10668000FD0182E3819384E011968C933196EF01B2
:10669000A1E7B9E002C08D91899329E0A537B2073F
:1066A000D1F786E3848384E085833696F093970957
:1066B000E0939609EF01ADE7B9E002C08D918993AF
:1066C00039E0A138B307D1F73496F0939709E093F6
:1066D00096092091960930919709D901E6E5F2E0F3
:1066E00002C081918D9382E0EC35F807D1F7C901A2
:1066F00006969093970980939609865E92400E9431
:106700005D2DDF91CF911F910F9108957F928F9210
:106710009F92AF92BF92CF92DF92EF92FF920F9330
:106720001F93CF93DF930E94FE370E943C3E5B0194
:106730006C0180E29EE4A0E0B0E0A80EB91ECA1E83
:10674000DB1E9924939404E0802E12E0712EF8C091
:1067500080918909813061F00E949637EC010097A1
:1067600009F4EEC00E942A2E892B09F0E9C00FC15E
:10677000C0E0D0E080918909833009F4C0C0843042
:1067800030F4813071F0823009F0D8C042C08530D9
:1067900009F4BDC0853008F4D3C0863009F0CEC0FE
:1067A000B6C081E799E062E972E00E9479358DE731
:1067B00099E062E972E00E9479350E943C3E7B01DB
:1067C0008C0160938A0970938B0980938C09909354
:1067D0008D090E943C3E8701FF24EE24E60EF71E41
:1067E000081F191FE0928A09F0928B0900938C0907
:1067F00010938D0981E061E00E94873270928909CF
:1068000010928E0910928F0910929009109291099E
:1068100097C0CE010E942C32823009F08FC081E7F0
:1068200099E066EF72E00E947935E6EDF3E08E01C3
:1068300004541D4FDF011196E180ED012196808106
:106840008630A1F0873030F4813051F0833009F088
:1068500049C009C0833369F0863309F043C03DC0A5
:1068600085E799E03CC089E799E039C081E899E083
:1068700036C02B8111966C9170E080E090E0962FED
:10688000882777276627620F711D811D911D298139
:1068900030E040E050E0A90133272227620F731F48
:1068A000841F951F2A8130E040E050E0542F432F91
:1068B000322F2227620F731F841F951F28EE33E0AB
:1068C00040E050E00E943A4160939209709393092E
:1068D000809394099093950905C08DE799E0BE01D6
:1068E0000E947935FE01EE0DF11DE017F10708F465
:1068F000A1CF83E060E00E94873283E01CC0CE011C
:106900000E942C328330D1F48092890907C0CE01D5
:106910000E942C32843069F4809389090E943C3EA5
:1069200060938E0970938F098093900990939109D9
:1069300007C0813029F48093890902C090928909A7
:1069400080918909843041F10E943C3E6A157B05A3
:106950008C059D0508F50E942237882389F3F8CE1F
:1069600080917909882321F089E799E00E94DA2C47
:1069700081E0DF91CF911F910F91FF90EF90DF9019
:10698000CF90BF90AF909F908F907F90089580910F
:10699000D3028131A9F6EECE0E94033880917109AD
:1069A0008823F1F6E6CFBC011092460286E492E01D
:1069B0004FE050E00E948E0681E0809389090E949A
:1069C00086330895CF93DF93DC01EB01722F632FA1
:1069D000822F932F9C01F90150E016C080819817F7
:1069E00071F431968081882371F411968C918D33E6
:1069F00031F4872F962F9C01F90151E004C0872FB5
:106A0000962F9C01F90111969C91992339F09032AF
:106A100029F09A3019F0552309F304C0513011F0D0
:106A200030E018C06A2F50E04150504002C0299316
:106A300011963A2F361B2C91222359F0203249F01F
:106A40002A3039F0263229F0832F90E084179507F9
:106A500074F31882832FDF91CF910895CF93DF9342
:106A6000FC01EC0137C08B3211F480E231C0853279
:106A700079F5DF0111969181392F30533A3070F05A
:106A8000892F8156863010F4375208C0892F8154DF
:106A9000863010F030E002C0392F3753FD013196B7
:106AA00011962C91922F90539A3070F0822F81562C
:106AB000863010F4975208C0822F8154863010F02F
:106AC00090E002C0922F9753832F8295807F892B6D
:106AD000899331968081882331F61882DF91CF9196
:106AE0000895DC01FB0186E001900D928150E1F7F1
:106AF00008959C01FB0180819181A281B381F901FC
:106B000080839183A283B383089581E08093DD091C
:106B10006093BA091092DB091092DC090895209164
:106B2000B90930E08091B809281B3109C9010895DD
:106B30004091B8098091B909481718F02FEF3FEF3D
:106B40000AC0E42FF0E0E856F64F8081282F30E0AD
:106B50004F5F4093B809C9010895E091B809809149
:106B6000B909E81718F0EFEFFFEF06C0F0E0E856BC
:106B7000F64F8081E82FF0E0CF010895089510923C
:106B8000E1091092E00988EE93E0A0E0B0E0809384
:106B9000E2099093E309A093E409B093E50982EA3E
:106BA00092E09093DF098093DE090895CF92DF92FF
:106BB000EF92FF920F931F93CF93DF937C016B01B2
:106BC0008A018091DD098823A1F0C0E0D0E00DC0EA
:106BD000D701ED91FC91D601AC0FBD1F0190F08162
:106BE000E02DC7016C9109952196C017D10780F35C
:106BF00004C0CB01642F0E94393CC801DF91CF91C2
:106C00001F910F91FF90EF90DF90CF900895DF9349
:106C1000CF930F92CDB7DEB7FC0169838091DD0978
:106C20008823C9F08091DC09803238F081E090E05F
:106C30009383828320E030E015C08091DB09E82F48
:106C4000F0E0E554F64F998190838F5F8093DB09E4
:106C50008093DC0905C0CE01019661E00E94393CB9
:106C600021E030E0C9010F90CF91DF91089580912C
:106C7000BA096BEB79E04091DC0921E00E94F63B18
:106C80001092DB091092DC091092DD09089541325F
:106C900008F040E2862F68E979E00E94BF3B10923D
:106CA000B8098093B90908950E9447360895109253
:106CB000B8091092B9091092DB091092DC090E9400
:106CC000CF3D0895762FF89465B121E030E040E0A3
:106CD00050E00090EC0904C0220F331F441F551FE1
:106CE0000A94D2F7922F9095962395B9972F9F717A
:106CF000982B9EBD0DB407FEFDCF1EBC0DB407FE44
:106D0000FDCF77FF04C01EBC0DB407FEFDCF8EB5CE
:106D100095B1292B25B978940895E42FF89475B18D
:106D200021E030E040E050E00090EC0904C0220F88
:106D3000331F441F551F0A94D2F7922F9095972323
:106D400095B96F71682B6EBD0DB407FEFDCFEEBD1A
:106D50000DB407FEFDCF85B1282B25B97894089591
:106D6000AC01FB01F89425B181E090E0A0E0B0E037
:106D70000090EC0904C0880F991FAA1FBB1F0A943A
:106D8000D2F7982F8095822385B98AE38EBD0DB402
:106D900007FEFDCF08C01EBC0DB407FEFDCF8EB5AB
:106DA00081934150504041155105A9F785B1982B69
:106DB00095B9789408951F93182F282F30E02076E6
:106DC00030708091ED0990E02817390799F080EA3A
:106DD0006FE143E00E948D36412F40764093ED09EC
:106DE00050E085E0559547958A95E1F780E86FE199
:106DF0000E948D361F9108951F93182F0E94DB3635
:106E000080E0612F0E9462361F9108950F931F93B7
:106E1000182F062F0E94DB3680E4612F402F0E943E
:106E20008D361F910F9108950F931F93182F072FE1
:106E30000E940637812F8F5F602F0E9406371F91B7
:106E40000F91089584ED61E10E94063782ED61E0C3
:106E50000E9406378AEE0E94FC3680FDFBCF82ED51
:106E600060E00E94063789ED0E94FC3690E096951E
:106E700087959695879581700895CF93DF93EC0160
:106E80000FC08CE10E94FC3681FF0AC080E86FE1F0
:106E900040E80E948D3680EA6FE140E80E948D361E
:106EA00080E06FE10E94623683FDEBCF82E060E01C
:106EB0007CE00E941437BE016050744F86E00E944F
:106EC00014378AE760E040E00E948D36F89425B1DF
:106ED00081E090E0A0E0B0E00090EC0904C0880FF1
:106EE000991FAA1FBB1F0A94D2F7982F809582235F
:106EF00085B98AE78EBD0DB407FEFDCFECEBF2E05D
:106F000007C080818EBD0DB407FEFDCF319621975D
:106F10002097B9F785B1982B95B9789480E86FE1FF
:106F200048E00E948D36DF91CF910895EF92FF9255
:106F30000F931F93DF93CF9300D000D000D0CDB735
:106F4000DEB789E30E94FC36882319F400E010E0E4
:106F500047C06091EE097091EF0980E00E941437FC
:106F600086E090E0BE016F5F7F4F0E94B036E980FF
:106F7000FA80F092EF09E092EE092B813C81E091DA
:106F8000EA09F091EB098D8187FD03C000E010E074
:106F90000EC0245030408F0101501040201731079F
:106FA00008F48901C8016CEB72E00E94B036F80168
:106FB000E454FD4F108281E0E8168CE0F80624F0DE
:106FC0008CE06FEF7BE005C00894E108F1088CE0ED
:106FD000B7010E94143780E86EE140E40E948D36CC
:106FE000C80126960FB6F894DEBF0FBECDBFCF9175
:106FF000DF911F910F91FF90EF90089588E361EB6F
:107000000E940637089588E360EB0E9406370895D2
:1070100084E061E00E94483F85E061E00E94483FD3
:1070200087E061E00E94483F86E060E00E94483FC0
:1070300084E061E00E94873F85E061E00E94873F35
:1070400085E060E00E94873F87E060E00E94873F24
:1070500080E58CBD8DB581608DBD0895CF93DF93A4
:10706000EB019093EB098093EA090CB406FC02C093
:107070000E94083884E08093EC09249A2C9A789432
:107080008FEF60E04FEF0E948D3662E070E080E0AD
:1070900090E00E944A3E80E06DE10E9462368823C3
:1070A000D1F31092EF091092EE0988E060E070E0F1
:1070B0000E9414378CE060E070E00E9414378AE090
:1070C0006FEF7BE00E94143784E060E07CE00E9478
:1070D000143786E06FEF71E10E9414370E94FE378B
:1070E00088E26FE370E30E94143780E369EF77EF83
:1070F0000E94143780EC6DE00E94063781EC60E05E
:107100000E94063780E862EC42E30E948D3686ECEE
:1071100062E17CE00E94143784EC62E10E94063751
:107120008AEC6CED75E00E94143784EE68810E9451
:10713000063785EE69810E94063782EE6A810E94D9
:10714000063783EE6B810E94063780EE6C810E94C9
:10715000063781EE6D810E94063784ED60E10E9462
:10716000063786ED60E071E00E9414378AEE0E94D7
:10717000FC3680FDFBCF8FE10E94DB3680E86BE1BF
:1071800040EC0E948D3680E86FE144E00E948D362D
:1071900082E70E94FC36863008F08F5FDF91CF9146
:1071A00008958F929F92AF92BF92CF92DF92EF920B
:1071B000FF920F931F93CF93DF937B018C01EA0122
:1071C0002CE330E040E050E00E948C416883C8012D
:1071D000B7012CE330E040E050E00E948C41122FD8
:1071E000032FF42EE52E622F732F842F952F2CE37F
:1071F00030E040E050E00E948C416983612F702FA5
:107200008F2D9E2D2CE330E040E050E00E948C4119
:10721000122F032FF42EE52E622F732F842F952F1C
:1072200028E130E040E050E00E948C416A83612F09
:10723000702F8F2D9E2D28E130E040E050E00E941D
:107240008C4179018A01C801B7016C5F7F4F8F4F74
:107250009F4F27E030E040E050E00E948C416F5F9C
:107260006B8320E0AA24BB24650101C02F5F822E1E
:107270009924F401EE54F84FCF0183709070892B5C
:1072800099F4CF0164E670E00E947941892B39F4CA
:10729000CF0160E971E00E947941892B29F48EE6E3
:1072A00091E0A0E0B0E004C08DE691E0A0E0B0E0A5
:1072B000A80EB91ECA1EDB1EC501A0E0B0E0E8168C
:1072C000F9060A071B0790F62E83F401EE54F84FD7
:1072D00083E0882E912C8E229F228114910499F4B0
:1072E000CF0164E670E00E947941892B39F4CF0127
:1072F00060E971E00E947941892B29F48EE691E0E2
:10730000A0E0B0E004C08DE691E0A0E0B0E0A81AF3
:10731000B90ACA0ADB0A980187010A191B092C0954
:107320003D09CF0164E670E00E9479417C01CF0104
:1073300060E971E00E947941AC01EEEAF2E060E0C0
:10734000613051F48114910449F4E114F10441F4E1
:107350004115510529F002C0808103C08CE101C0B4
:107360008DE190E0A0E0B0E0081719072A073B077D
:1073700040F0081B190B2A0B3B0B6F5F31966C30EA
:10738000F9F66F5F6D83802F8F5F8C83DF91CF91D4
:107390001F910F91FF90EF90DF90CF90BF90AF9033
:1073A0009F908F900895EF92FF920F931F937B0110
:1073B0008C018091070A9091080AA091090AB09166
:1073C0000A0AE816F9060A071B0771F0C801B70197
:1073D0004CEF59E00E94D138E092070AF092080A77
:1073E0000093090A10930A0A1F910F91FF90EF90E2
:1073F00008950E94D3392091020A30E02E54384F6C
:10740000C90108950E94D3398091010A90E008953E
:107410000E94D3398091FF0990E008950E94D339EA
:107420008091000A90E008950E94D3398091FD096F
:1074300090E008950E94D3398091FE0990E008956C
:107440004F925F926F927F928F929F92AF92BF9274
:10745000CF92DF92EF92FF920F931F93CF93DF9320
:107460004C01DC0116961C91612F70E080E090E0E9
:1074700020E833E341EE51E00E943A415B016C01A8
:1074800022EB37E0E12FF0E0EE54F84F1DC0C901C8
:1074900083709070892BB1F4C90164E670E00E949A
:1074A0007941892B39F4C90160E971E00E94794181
:1074B000892B41F480E891E5A1E0B0E0A80EB91E67
:1074C000CA1EDB1E2F5F3F4F2E173F0701F7D40167
:1074D00015968C91482E5524C90164E670E00E94EF
:1074E00079417C01C90160E971E00E9479418C0118
:1074F000C1E0D0E093E0692E712C6222732227C094
:10750000C230D10591F46114710479F4E114F104ED
:1075100019F40115110549F480E89BE3A6E2B0E0F7
:10752000A80EB91ECA1EDB1E11C0FE01E355FD4F99
:10753000608170E080E090E020E831E541E050E0DB
:107540000E943A41A60EB71EC81ED91E2196C41528
:10755000D505B4F2D40112966C9170E080E090E011
:1075600020E13EE040E050E00E943A417B018C0186
:10757000F401618170E080E090E02CE330E040E0D5
:1075800050E00E943A41E60EF71E081F191FD40171
:107590008C91E80EF11C011D111D14966C9170E088
:1075A00061507040882777FD8095982F20E831E55D
:1075B00041E050E00E943A41E60EF71E081F191FF5
:1075C000EA0CFB1C0C1D1D1DB701C801DF91CF91FA
:1075D0001F910F91FF90EF90DF90CF90BF90AF90F1
:1075E0009F908F907F906F905F904F9008956093E1
:1075F0006002709361028093620290936302089527
:107600006093F2097093F3098093F4099093F5095C
:1076100020916002309161024091620250916302B8
:10762000260F371F481F591F2093F6093093F7097B
:107630004093F8095093F90982E090E09093FB0998
:107640008093FA090E943C3E6093030A7093040AF7
:107650008093050A9093060A0895EF92FF920F9384
:107660001F931CC02F5F3F4F4F4F5F4F2093F20976
:107670003093F3094093F4095093F50988EE93E0B1
:10768000A0E0B0E0E80EF91E0A1F1B1FE092030AFB
:10769000F092040A0093050A1093060A0E943C3EE9
:1076A000E090030AF090040A0091050A1091060A7E
:1076B0006E197F09800B910B2091F2093091F3092B
:1076C0004091F4095091F509685E73408040904004
:1076D00048F68091F6099091F709A091F809B091C8
:1076E000F909281739074A075B07E8F0E091F00924
:1076F000F091F1093097B9F009956115710581058F
:10770000910519F00E94003B0EC020E030E080910E
:10771000FA099091FB09892B11F021E030E03093B8
:10772000FB092093FA096091F2097091F3098091A5
:10773000F4099091F5091F910F91FF90EF90089532
:107740009093F1098093F0098091F2099091F309E7
:10775000A091F409B091F5098093F6099093F70987
:10776000A093F809B093F9090E942D3B08950E9457
:107770002D3B0E94D3398091FF0990E00895982F06
:10778000413210F040E030C080910B0A8823E1F7CD
:1077900081E080930B0A8FEF8093760A1092310A72
:1077A00041504093320A4F5F990F916090930C0AB9
:1077B00085EE8093BC0080910B0A8130E1F38091CB
:1077C000310A841710F44091310A20E030E00AC0F9
:1077D000FB01E20FF31FD901AF5EB54F8C9180839F
:1077E0002F5F3F4F2417A0F3842F08951F93582F26
:1077F000122F413210F081E03AC080910B0A8823A9
:10780000E1F782E080930B0A8FEF8093760A109263
:10781000310A4093320AA1E1BAE0FB0102C0819132
:107820008D938E2F861B8417D0F3852F90E0880FC1
:10783000991F80930C0A85EE8093BC00112321F0E0
:1078400080910B0A8230E1F38091760A8F3F11F428
:1078500080E00DC08091760A803211F482E007C08A
:107860008091760A803311F084E001C083E01F919B
:107870000895482F613210F081E0089580910B0A3D
:10788000843011F082E008956093540AA3E3BAE0D3
:10789000842F9C01F90102C081918D938E2F841B4E
:1078A0008617D0F380E008951F920F920FB60F92C3
:1078B00011242F933F934F935F936F937F938F93F5
:1078C0009F93AF93BF93EF93FF938091B90090E0A4
:1078D000887F90708036910509F4DCC0813691056F
:1078E000CCF58832910509F47BC089329105B4F456
:1078F0008031910509F46FC0813191053CF4009706
:1079000009F431C1089709F039C165C08831910582
:1079100009F466C0809709F031C17DC080349105BB
:1079200009F49FC08134910544F48033910509F432
:107930007DC0C89709F022C184C08035910509F443
:1079400084C08835910509F491C08834910509F007
:1079500015C198C08839910509F4FDC08939910590
:10796000ECF48837910509F495C0893791054CF4FA
:107970008836910509F48EC08037910509F0FEC064
:1079800089C08838910509F4E6C08039910509F469
:1079900087C08038910509F0F1C082C0803B910515
:1079A00009F4B0C0813B91054CF4803A910509F48B
:1079B00089C0883A910509F0E1C0A4C0803C9105D6
:1079C00009F4CDC0883C910509F4C9C0883B9105F4
:1079D00009F0D4C0ACC080910C0A8093BB00B9C040
:1079E0009091310A8091320A981768F49091310A87
:1079F000E92FF0E0EF5EF54F80818093BB009F5F41
:107A00009093310AA6C085ED8093BC008091BC00A4
:107A100084FDFCCFB1C080E28093760A85ED80932F
:107A2000BC008091BC0084FDFCCFA6C080E38093A5
:107A3000760A85ED8093BC008091BC0084FDFCCF6C
:107A40009BC088E38093760A8AC08091310A909126
:107A5000BB00E82FF0E0EF5EF54F90838F5F8093DF
:107A6000310A9091310A8091320A71C08091310AB5
:107A70009091BB00E82FF0E0EF5EF54F90838F5FB1
:107A80008093310A85ED8093BC008091BC0084FD19
:107A9000FCCF72C083E080930B0A1092750A59C024
:107AA0008091750A803208F056C08091750A9091D5
:107AB000BB00E82FF0E0EB5AF54F90838F5F809387
:107AC000750A47C08091750A803230F4E091750ADA
:107AD000F0E0EB5AF54F108285ED8093BC00809169
:107AE000BC0084FDFCCF10920B0A6091750AE091F6
:107AF0000F0AF091100A85E59AE070E0099510925E
:107B0000750A2DC084E080930B0A1092530A1092DC
:107B1000540AE0910D0AF0910E0A09958091540AD9
:107B2000882329F481E08093540A1092330A9091BB
:107B3000530AE92FF0E0ED5CF54F80818093BB00A4
:107B40009F5F9093530A9091530A8091540A98171B
:107B500010F485EC01C085E88093BC000FC085EC73
:107B60008093BC0009C01092760A85ED8093BC001A
:107B70008091BC0084FDFCCF10920B0AFF91EF9125
:107B8000BF91AF919F918F917F916F915F914F9135
:107B90003F912F910F900FBE0F901F90189510924C
:107BA0000B0A81E161E00E94873F80E161E00E9471
:107BB000873FE9EBF0E080818E7F808380818D7F3D
:107BC000808380E28093B80085E48093BC000895B0
:107BD0001F920F920FB60F9211242F933F934F9342
:107BE0005F936F937F938F939F93AF93BF932091F6
:107BF0007B0A30917C0A40917D0A50917E0A7091F7
:107C00007F0ADA01C9010296A11DB11D672F6A5FC3
:107C10006D3730F06D57DA01C9010396A11DB11D12
:107C200060937F0A80937B0A90937C0AA0937D0ADD
:107C3000B0937E0A8091770A9091780AA091790A90
:107C4000B0917A0A0196A11DB11D8093770A909395
:107C5000780AA093790AB0937A0ABF91AF919F9165
:107C60008F917F916F915F914F913F912F910F90E5
:107C70000FBE0F901F9018958FB7F89420917B0A34
:107C800030917C0A40917D0A50917E0A8FBFB901E4
:107C9000CA0108959B01AC017FB7F8948091770ADF
:107CA0009091780AA091790AB0917A0A66B5A89B5A
:107CB00005C06F3F19F00196A11DB11D7FBFBA2FFE
:107CC000A92F982F8827860F911DA11DB11D63E054
:107CD000880F991FAA1FBB1F6A95D1F7BC012DC041
:107CE000FFB7F8948091770A9091780AA091790A69
:107CF000B0917A0AE6B5A89B05C0EF3F19F001964E
:107D0000A11DB11DFFBFBA2FA92F982F88278E0F55
:107D1000911DA11DB11DE3E0880F991FAA1FBB1F74
:107D2000EA95D1F7861B970B885E9340C8F22150E5
:107D300030404040504068517C4F2115310541058D
:107D4000510571F60895019739F0019729F0880FD0
:107D5000991F01970197F1F70895789484B582608F
:107D600084BD84B5816084BD85B5826085BD85B5DF
:107D7000816085BDEEE6F0E0808181608083E1E88E
:107D8000F0E01082808182608083808181608083C6
:107D9000E0E8F0E0808181608083E1EBF0E08081C9
:107DA00084608083E0EBF0E0808181608083EAE79B
:107DB000F0E0808184608083808182608083808124
:107DC000816080838081806880831092C1000895E3
:107DD0001F93CF93DF93182FEB0161E00E94483F80
:107DE000209709F44AC0CF3FD10509F449C0E12FDB
:107DF000F0E0E45EF34F84918330C1F0843028F4E6
:107E0000813051F08230B1F50CC0863019F18730E5
:107E100049F1843079F514C084B5806884BDC7BD4C
:107E200033C084B5806284BDC8BD2EC080918000FF
:107E3000806880938000D0938900C093880024C01C
:107E400080918000806280938000D0938B00C093EB
:107E50008A001AC08091B00080688093B000C093FF
:107E6000B30012C08091B00080628093B000C093D4
:107E7000B4000AC0C038D1051CF4812F60E002C0F4
:107E8000812F61E00E94873FDF91CF911F9108957C
:107E9000CF93DF93482F50E0CA018450944FFC01E8
:107EA00034914452544FFA018491882369F190E04F
:107EB000880F991FFC01E254F44FA591B491FC0185
:107EC000E853F44FC591D491662351F42FB7F89439
:107ED0008C91932F909589238C93888189230BC053
:107EE000623061F42FB7F8948C91932F9095892389
:107EF0008C938881832B88832FBF06C09FB7F8940B
:107F00008C91832B8C939FBFDF91CF910895482F45
:107F100050E0CA01845E934FFC012491CA01845051
:107F2000944FFC0194914452544FFA0134913323FD
:107F300009F440C0222351F1233071F0243028F499
:107F40002130A1F0223011F514C02630B1F02730D5
:107F5000C1F02430D9F404C0809180008F7703C031
:107F6000809180008F7D8093800010C084B58F77D2
:107F700002C084B58F7D84BD09C08091B0008F7729
:107F800003C08091B0008F7D8093B000E32FF0E0BC
:107F9000EE0FFF1FE853F44FA591B4912FB7F8945B
:107FA000662321F48C919095892302C08C91892BB2
:107FB0008C932FBF0895682F70E0CB01845E934FA0
:107FC000FC012491CB018450944FFC0144916452F4
:107FD000744FFB019491992319F420E030E03CC0E8
:107FE000222351F1233071F0243028F42130A1F004
:107FF000223011F514C02630B1F02730C1F0243002
:10800000D9F404C0809180008F7703C080918000F4
:108010008F7D8093800010C084B58F7702C084B5B7
:108020008F7D84BD09C08091B0008F7703C080919F
:10803000B0008F7D8093B000892F90E0880F991F4A
:108040008E52944FFC01A591B4918C9120E030E0C8
:10805000842311F021E030E0C9010895CF93DF932C
:108060000E94AD3E0E94551CC0E0D0E00E94F21C70
:108070002097E1F30E940000F9CFCF92DF92EF92B8
:10808000FF920F931F93CF93DF937C016B018A01C3
:10809000C0E0D0E00FC0D6016D916D01D701ED9128
:1080A000FC910190F081E02DC7010995C80FD91FFF
:1080B000015010400115110571F7CE01DF91CF91EC
:1080C0001F910F91FF90EF90DF90CF900895DC010A
:1080D000ED91FC910190F081E02D09950895CF93E9
:1080E000DF93DB010D900020E9F71197A61BB70B7A
:1080F000EC01E881F9810280F381E02DAD01099561
:10810000DF91CF9108954F925F927F928F929F92CD
:10811000AF92BF92CF92DF92EF92FF920F931F9395
:10812000DF93CF93CDB7DEB7A1970FB6F894DEBF3C
:108130000FBECDBF2C01742ECB01223008F42AE0F3
:1081400019A231E2C32ED12CCC0EDD1E822E992431
:10815000AA24BB24672D752FA50194010E948C4190
:1081600079018A01C801B701A50194010E943A4131
:10817000472D461B0894C108D1084A3014F4405DCD
:1081800001C0495CF6014083E114F10401051105C9
:1081900021F07E2C5F2DC801DDCFC201B6010E9407
:1081A0006F40A1960FB6F894DEBF0FBECDBFCF9142
:1081B000DF911F910F91FF90EF90DF90CF90BF90D4
:1081C000AF909F908F907F905F904F900895CF9247
:1081D000DF92EF92FF920F931F93CF93DF93EC0107
:1081E0006A017B012115310541F4E881F981019093
:1081F000F081E02D642F09951FC02A303105D1F49C
:1082000077FF17C0E881F9810190F081E02D6DE2E0
:1082100009958C0144275527BA014C195D096E094F
:108220007F09CE012AE00E9483409801280F391F60
:1082300004C02AE00E9483409C01C901DF91CF91D4
:108240001F910F91FF90EF90DF90CF900895EF92E4
:10825000FF920F931F937B019A010027F7FC009573
:10826000102FB801A7010E94E7401F910F91FF90C6
:10827000EF900895629FD001739FF001829FE00DFF
:10828000F11D649FE00DF11D929FF00D839FF00D95
:10829000749FF00D659FF00D9927729FB00DE11D41
:1082A000F91F639FB00DE11DF91FBD01CF0111241E
:1082B0000895991B79E004C0991F961708F0961B42
:1082C000881F7A95C9F780950895AA1BBB1B51E1B9
:1082D00007C0AA1FBB1FA617B70710F0A61BB70B36
:1082E000881F991F5A95A9F780959095BC01CD01DB
:1082F000089597FB092E07260AD077FD04D0E5DF05
:1083000006D000201AF4709561957F4F0895F6F716
:10831000909581959F4F0895A1E21A2EAA1BBB1B31
:10832000FD010DC0AA1FBB1FEE1FFF1FA217B30741
:10833000E407F50720F0A21BB30BE40BF50B661F57
:10834000771F881F991F1A9469F76095709580951B
:1083500090959B01AC01BD01CF010895EE0FFF1F69
:108360000590F491E02D09942F923F924F925F92E5
:108370006F927F928F929F92AF92BF92CF92DF9235
:10838000EF92FF920F931F93CF93DF93CDB7DEB79A
:10839000CA1BDB0B0FB6F894DEBF0FBECDBF09942E
:1083A0002A88398848885F846E847D848C849B8485
:1083B000AA84B984C884DF80EE80FD800C811B8193
:1083C000AA81B981CE0FD11D0FB6F894DEBF0FBEC2
:0A83D000CDBFED010895F894FFCF32
:1083DA0074007077006C6F63006E7077006370775B
:1083EA00007069640064006D007900763D5B00727C
:1083FA00736E0072627400656E006D6D00726400C7
:10840A00743D5B006F70656E646F6F7200426F73CC
:10841A00746F6E2C4D41006F70656E737072696E69
:10842A006B6C6572000069692D3000CC0936777B68
:10843A007201DA197501F9167801F2127B01F51742
:10844A007E018C18810189158401AE0987014110CA
:10845A008A01B10D8D01561790017A0F930181118E
:10846A00960142089901D31A9C01560FC800B9080F
:10847A0000206CC708030101D208010101DC0801D0
:10848A00C0FFE60801A8FFF2080101FFF70801167C
:10849A00FFFC0801C0FF010901A8FF0E090101FF45
:1084AA0013090101FF18090150FF1D090200FF28E5
:1084BA0009020101290901000539090301014609D7
:1084CA000300F05209030008610903003C71090323
:1084DA003C787F090300018E090301019F090364A7
:1084EA00FAAE09030AF0BE09010001CD090300FF33
:1084FA00DE09016EFFE90901C8FFF709010001065B
:10850A000A01110A150A190A1D0A210A250A290A45
:10851A000100010A500041726475696E6F2D303096
:10852A000000000000003703010306FF6382536363
:10853A00100E00000000000057073D406F000000C9
:10854A00002E6F4F001408150105051500000000E4
:10855A00F7283D400000400014005400FFFFFFFFD1
:10856A00FFFF000000000000FFFFFFFFFFFF000009
:10857A0000000736D6358F359835AD35BE351F1C08
:0A858A001F1E1F1E1F1F1E1F1E1FB5
:00000001FF
